:100000000C9464160C948C160C948C160C948C1610
:100010000C948C160C948C160C948C160C948C16D8
:100020000C948C160C948C160C949F300C941131FB
:100030000C948C160C948C160C948C160C948C16B8
:100040000C948C160C948C160C948C160C948C16A8
:100050000C948C160C948C160C948C160C949E2874
:100060000C948C160C948C160C948C160C948C1688
:100070000C948C160C948C160C948C160C948C1678
:100080000C9496290C948C160C948C160C948C164B
:100090000C948C160C948C160C948C160C948C1658
:1000A0000C948C160C948C160C948C16080800007A
:1000B000000000000000000030002010000004805C
:1000C000000020000200081408E2451228100C0E5F
:1000D0006AF6B09060001EB3DFDFB3935F0E00CF0F
:1000E000300304186483AA15BF007F43404040409A
:1000F000407F00BF15AA3FBF20A120A020A020A0C4
:1001000020A020A03FBF6DFBBF57EDBDDBEE8040C0
:100110006080640CF040092A12242748B3CC3C08C4
:10012000C4B6249248178E556892640CF142092A8D
:1001300012242748B3CC0000000000403FFFB0531A
:100140006C82640CF1423F08C4B6249248037EE1FD
:100150005C423925510A3D7F8000000000003E08C6
:10016000C4B4209000005EE15C423925510A00F8D9
:1001700004E6A26202C220075409A80950130686A9
:10018000868C1CF8F0005017A223A07F7F00AA5491
:10019000FE02FA0A0A0A0A0A0AFA02FE54AAFEFE35
:1001A000062686462606060606060606FEFE6FDFBD
:1001B000B8B7B7B7B7B7B7B7B7B7B7B7B7B7B7B7CE
:1001C000B7B7B7B8DF6FFFFFFFFFFF00FFFFE3E345
:1001D000E3E3C307FEFCE3E3E3E3E3E3E3E3FCFE83
:1001E00007C3E3E3E3E3FFFF00FFFFFFFFFF0000C0
:1001F000000000000000001C3800180C0000048003
:1002000000002000020010281245E2081408020E27
:10021000162A24283000025020102E0E0C00000652
:1002200088FFF76B8C02ACEECE003F7F7F7FFFFB39
:10023000F3FF00AEEEEA6EEEE06F68E8E8EFC3DCD5
:10024000D0E8AFA0EACEA64CD1EFD1AB6CA6081196
:10025000261C0A503065040CCB4938303432A29247
:10026000042811E39A04B2E1E3E6CCF87FF0081029
:1002700010337FDEBFFF000080E038BF5D3E80644A
:100280001C18FF20106C70EB7CC6E371188CFFBF4C
:10029000DF391C0E0301DE1D7FB860C080003269AB
:1002A000C44034100E0186C3407C22221008048012
:1002B0000030303060FE20005000A000403FFE6063
:1002C000C0C0C00002007F808000A0000200EFEFED
:1002D000AD01F3FBFBFAE202E6F602F6ECEEE6EE27
:1002E00003FB0A0A0BFB1313130BFB03CEEC7E7FFD
:1002F0003F007FFF1F007E7F3B006FFFFB00007F02
:100300007F07001F7F7F00DFF73C00FBEF3F00F31C
:10031000FFFE00F8DE8CFECEFF003FFEFF00FC7EFD
:10032000FF00FCFFE7007FFFE7003FFDF700000054
:10033000000000000000000008100030080000026B
:10034000002000000004102810000008140800001D
:100350001028243830001C1E36723E721C0054A334
:1003600014A95E0BD02AFF6F10FF90EF81FE90EF73
:1003700081FE90FF00FE10EF00DF10B010D01FD004
:1003800010B010DF01FE7FF6DF7AFCBEEB46207076
:100390004C40902840800502824E31405049000078
:1003A0000050BC00107FC6F8E0AE53F0B89E0000CD
:1003B000010307FFF9F60080C040E0F07B3FC0C0BA
:1003C000601008040402030100008080C3E4EE070B
:1003D0000703010000005F7FF0C080000000800084
:1003E0000E90A0C000007C331018180F040220608B
:1003F0004EF060028CF00001022183C776B9389C70
:100400008794E0C0A004FF7C832100000004FEEE7E
:1004100010FC14EC04FC14EC04FC14FC00FE10EEC4
:1004200000F6101A1016F016101A10F600FEFFFF54
:10043000C0D5D9D5D5D5E6D5D5D5D9D5D5D5E6D557
:10044000D5D5D9D5D5FF66555555995555FF65551F
:100450005555995555FF6555555599555555FFFFB6
:10046000015599555555FFFF005599555555101093
:100470000000C020F010F010F010F020C08000004C
:1004800000003F203F203F203F203F203F10000042
:100490000000000000000000000000FCFC00000064
:1004A00000000000000000000000003F3F000000CE
:1004B000000000000000000000000000000000003C
:1004C000000018181818181818181818181800000C
:1004D000000000FCFC000000000000000000000024
:1004E0000000003F3F00000000000000000000008E
:1004F0001010FFFFFFFFFFFFFFFFFFFFFFFFFFFFEA
:10050000FFFFFFFFFFFFFFFFFFFFFFFFFFFFFFFFFB
:10051000FFFF080800080C7E7E0C0800000203BFE5
:10052000BF0302000080C0E7E7C08000002030F970
:10053000F9302000001818187E3C18001800181810
:1005400018187E3C7E3C18000018181818187E3CBD
:10055000180000180010307E7E3010000040C0FDF2
:10056000FDC04000000103E7E703010000040C9F09
:100570009F0C040000183C7E181818003C7E1818C8
:10058000181800181818180000183C7E18000018D9
:100590003C7E18180808FFFFFFFFFFFFFFFF080859
:1005A0003C7E66FFDBFFBDFFBDFFDBFF66FF3C7EE1
:1005B000003C3C7E42FFBDFFC3FF7EFF3C7E003C13
:1005C0000000007E7EFFDBFFFFFF7EFF007E00005D
:1005D0000000000000FFFFFFFFFF00FF0000000021
:1005E0000000007E7EFFFFFFDBFF7EFF007E00003D
:1005F000003C3C7E7EFFC3FFBDFF42FF3C7E003CD3
:100600001E3F317F61FFC2FFC2FF61FF317F1E3F8E
:10061000001E1E3F21FFC2FFE1FF3FFF1E3F001EE5
:100620000000003E3EFFC3FFFFFF3EFF003E000014
:100630000000000000FFFFFFFFFF00FF00000000C0
:100640000000003E3EFFFFFFC3FF3EFF003E0000F4
:10065000001E1E3F3FFFE1FFC2FF21FF1E3F001EA5
:100660001C10000000F8F8FC04FE02FFFAFF22FF55
:1006700022FFFAFF02FFFAFFAAFFAAFF8AFF02FF8A
:10068000FAFF82FF82FF82FF02FFFAFF2AFF2AFFA2
:100690003AFF02FF04FEF8FC00F80006060F091FEF
:1006A000040F0207020702070207020702070207F8
:1006B00002070207020702070207020702070207F2
:1006C00002070207020702070207020701030001EF
:1006D0000000101004C62E1FEFDE4FD7DE6FE7DEDE
:1006E0003C10E00000000D0C615B52A3A3525B6163
:1006F0000C0D0000088C5C3EDEBC9EAEBCDECEBCA9
:100700007820C00000010C0C635754A7A75457630E
:100710000C0C0100088C5C3EDEBC9EAEBCDECEBC88
:100720007820C00000011818435755A7A755574314
:100730001818010004C62E1FEFDECFD7DEEFE7DE6C
:100740003C10E00000001918415B53A3A3535B4128
:10075000181900000000C082DEDC1EDEDE1EDCDEBA
:1007600082C0000000000C0C31BBBB3131BBBB317F
:100770000C0C000000008004BCB83CBCBC3CB8BC05
:100780000480000000000D0D31B7B63333B6B73129
:100790000D0D000000008004BCB8BCBCBCBCB8BCE3
:1007A000048000000000191923B7B63333B6B7230D
:1007B000191900000000C082DEDCDEDEDEDEDCDED9
:1007C00082C000000000181821BBBB3131BBBB2127
:1007D0001818000000000070B0C46CDCD26CCCB003
:1007E000700000000000000C0DC3EA2B2BEAC30DC3
:1007F0000C000000000000E06088D8B8A4D8986021
:10080000E00000000000000C0DC3E42727E4C30D46
:100810000C000000000000E06088D8B8A4D8986000
:10082000E0000000000000181BC7E52727E5C71BF4
:100830001800000000000070B0C4ECDCD2ECCCB0BA
:10084000700000000000001819C3EB2B2BEBC3193C
:10085000180000000000E04034D4D63636DAD83430
:1008600048E0000000000C0C614A5A13135A4A6118
:100870000C0C00000000C08068A8AC6C6CB4B068C0
:1008800090C0000000000D0C6245550606554562FB
:100890000C0D00000000C08068A8AC6C6CB4B0689F
:1008A00090C0000000001918424555060655454203
:1008B000181900000000E04034D4D63636DAD834B7
:1008C00048E0000000001818414A5A13135A4A41E0
:1008D0001818000000000030DCEE36EAEE34EEDCE2
:1008E000300000000000080D327D797979797D3281
:1008F0000D08000000000060B8DC6CD4DC68DCB8D7
:10090000600000000000080C317B727373727B3151
:100910000C08000000000060B8DCECD4DCE8DCB8B7
:10092000600000000000101A217B727373727B213B
:100930001A10000000000030DCEEF6EAEEF4EEDC07
:100940003000000000001019247D797979797D2428
:10095000191000001010DEFFFFFFFFFFFFFFFFFF79
:10096000FFFFFEFCF0E0013F3F7FFFFFFFFFFFFFC7
:10097000FFFF7F3F3F0300C0F6FFFFFEFFFFFFFFCB
:10098000FEFFFFF6C000001D3F7FFFFFFF7F7FFFE0
:10099000FFFF7F3F1D000000F0F8FCFEFFFFFFFEA1
:1009A000FEFCF8F0000000001C3F7FFFFF7F7FFF90
:1009B000FF7F3F1C000000E0F0FCFEFEFFFFFFFF9A
:1009C000FEFEFCF8E000001D3F7FFFFFFF7F7FFF82
:1009D000FFFF7F3F1D00000070FCFEFFFFFFFFFFD9
:1009E000FFFEFC700000001C3F3F7FFFFFFFFFFF8A
:1009F000FF7F3F3F1C001010004CFE3E7EE6C6FE0F
:100A0000740870F0E0C000000000010E527B6B61C2
:100A10000C1F3CA3DFF720000026FF1F3FF3E3FF7E
:100A20003A8438F8F0E000000000000F11050DB026
:100A3000F6EFDC110F1B10000080E0F030F88800AA
:100A4000F0E2337FFEC6CE3C00372F001F2F270079
:100A500080F9F20203596C000000C0E060F0100061
:100A6000E0C466FEFC8C9C78006F5F010EE7F380AB
:100A70000103547407B3D90010107EFFFFFFFFFF7E
:100A8000FFFFFFFEFCFCF8F0E00000010F5FFFFF3E
:100A9000FFFFFFFFFFFFFFFFFF3080E0F0F8F8FCF3
:100AA000FCF8FEFFFFFFFFFFFFFE7FFFFF7FFFFF62
:100AB000FFFFFFFFFFFFFFFFFFFD10100000808022
:100AC000803C6767AFB9B99F4B8C000000030103FE
:100AD000B9DDBC0B091BBDDDE30300000000808015
:100AE000803C6767AFB9B99F4B8C000000030103DE
:100AF00001BDDCAB011B9DEDD30300000000808035
:100B000080BC27A7CFD9D99FCB8C0000000301035D
:100B1000011CBCC11C1DECE0010100000080C0C034
:100B2000C05C33B3D7DCDC97DB9A00000001000126
:100B300000001CA1DC1DECE00101000000C060E031
:100B4000405C39B1D3DFDC9CDB9A00000000000080
:100B50000C5D6C35001D1CECE10100000080C0C084
:100B600080BC6667AFB9B9BF579800000001001993
:100B7000BCDCB403011BBDDDE3030000000080808A
:100B800000709E9E32727E6EB61000000003113B14
:100B9000B9DDA8061337BBDBE2030000000000004C
:100BA00000709E9E32727E6EB61000000006031723
:100BB000B9DDA8060337BBDBE2030000008C4B9FC6
:100BC000B9B9AF67673C8080800000000003E3DDB7
:100BD000BD1B090BBCDDB90301030000008C4B9F5A
:100BE000B9B9AF67673C8080800000000003D3ED97
:100BF0009D1B01ABDCBD010301030000008CCB9FFA
:100C0000D9D9CFA727BC808080000000000101E077
:100C1000EC1D1CC1BC1C010301030000009ADB9702
:100C2000DCDCD7B3335CC0C0C0800000000101E051
:100C3000EC1DDCA11C00000100010000009ADB9CFF
:100C4000DCDFD3B1395C40E060C000000001E1ECC2
:100C50001C1D00356C5D0C0000000000009857BFA3
:100C6000B9B9AF6766BC80C0C08000000003E3DD97
:100C7000BD1B0103B4DCBC19000100000010B66EFE
:100C80007E72329E9E700080800000000003E2DBD6
:100C9000BB371306A8DDB93B110300000010B66E88
:100CA0007E72329E9E700000000000000003E2DBB6
:100CB000BB370306A8DDB917030600001010C0E01B
:100CC000F0F0FCFFFFFFFFFFFFFFFFFF9E00071F8D
:100CD0003FFFFFFFFFFFFFFFFFFFFFF703009EFF48
:100CE000FFFFFFFFFFFFFFFFFCF0F0E0C00003F796
:100CF000FFFFFFFFFFFFFFFFFFFF3F1F070002088F
:100D0000030310100E070F3ABC3EDECEBEBE3EBC43
:100D10003A0F070E000000000D1A53136BBBBA7593
:100D2000180000001E0F071DDE1FEFE7DFDF1FDECC
:100D30001D070F1E00000000366D6909355D5D3A24
:100D40000C0000000E070F3ABC3EDECEBEBE3EBC1D
:100D50003A0F070E000000006D5A13136BBBBA75F3
:100D6000180000001E0F071DDE1FEFE7DFDF1FDE8C
:100D70001D070F1E00000000366D6909355D5D3AE4
:100D80000C00000000000C3E3FCFDEBE3EBEBC7E2D
:100D9000770F070E006090B87B136B6B2A331D0032
:100DA000000000000000061F9FE7EFDF1FDFDE3FAF
:100DB0003B070F1E0030485C3D09155555590E0084
:100DC0000000000000000C3E3FCFDEBE3EBEBC7EF9
:100DD000770F070E006090B87B132B2B2A335D60D2
:100DE000000000000000061F9FE7EFDF1FDFDE3F6F
:100DF0003B070F1E0030485C3D09155555590E0044
:100E0000000000000000003CCE1EBEBE7E7E7E7B49
:100E10000707030618243C3C436A2B331A4D000095
:100E2000000000000000001EE70FDFDF3FBF3E3B79
:100E300007070E000C121E1E011555596D06000005
:100E4000000000000000003CCE1EBEBE7E7E7E7B09
:100E50000707030618243C3C432A2B335A6D4000F5
:100E6000000000000000001EE70FDFDF3FBF3E3B39
:100E700007070E000C121E1E011555596D060000C5
:100E80000000000000000038DC3C76EEEEECC2FE14
:100E9000FE0E0C0000000E1C1B52590415450901E2
:100EA000000000000000001CEE1EB36FEFDDC3FE6B
:100EB0007E0E1C000000070E0D296C420A220C0059
:100EC0000000000000000038DC3C76EEEEECC2FED4
:100ED000FE0E0C0000000E1C5B5219041565690122
:100EE000000000000000001CEE1EB36FEFDDC3FE2B
:100EF0007E0E1C000000070E0D296C420A220C0019
:100F0000000000001C0E1EDEECFEFEFEFEFEFEECEF
:100F1000DE1E0E1C000000050B2305656565230B16
:100F2000050000003C1E1EE6FFFFFFFFFFFFFFFF66
:100F3000E61E1E3C0000000205112A0A6A723105F5
:100F4000020000001C0E1EDEECFEFEFEFEFEFEECAD
:100F5000DE1E0E1C000000050B6365551525230BD6
:100F6000050000003C1E1EE6FFFFFFFFFFFFFFFF26
:100F7000E61E1E3C0000000205112A0A6A723105B5
:100F800002000000000C0EFEFEC2ECEEEE763CDC31
:100F90003800000000000000010945150459521BEB
:100FA0001C0E0000001C0E7EFEC3DDEF6FB31EEEB4
:100FB0001C00000000000000000C220A426C290DF9
:100FC0000E070000000C0EFEFEC2ECEEEE763CDCDE
:100FD0003800000000000000016965150419525B2B
:100FE0001C0E0000001C0E7EFEC3DDEF6FB31EEE74
:100FF0001C00000000000000000C220A426C290DB9
:101000000E070000060307077B7E7E7EBEBE1ECE57
:101010003C0000000000000000004D1A332B6A4322
:101020003C3C2418000E07073B3EBF3FDFDF0FE7C5
:101030001E000000000000000000066D595515015B
:101040001E1E120C060307077B7E7E7EBEBE1ECED2
:101050003C0000000000000000406D5A332B2A4382
:101060003C3C2418000E07073B3EBF3FDFDF0FE785
:101070001E000000000000000000066D595515011B
:101080001E1E120C0E070F777EBCBE3EBEDECF3F8B
:101090003E0C000000000000001D332A6B6B137B28
:1010A000B89060001E0F073B3FDEDF1FDFEFE79FBA
:1010B0001F06000000000000000E59555515093D9F
:1010C0005C4830000E070F777EBCBE3EBEDECF3FD1
:1010D0003E0C000000000000605D332A2B2B137BC8
:1010E000B89060001E0F073B3FDEDF1FDFEFE79F7A
:1010F0001F06000000000000000E59555515093D5F
:101100005C48300010103F1F7FFFFFFFFFFFFFFF15
:10111000FFFFFF7F1F3F0000007FFFFFFFFFFFFF7C
:10112000FFFF7F1C0000000E7FFFFFFFFFFFFFFFA0
:10113000FFFFFFFF1F3F70F8FCFFFFFFFFFFFFFFF8
:10114000FFFF6000000000003EFFFFFFFFFFFFFF0A
:10115000FFFF7F0F1F1F3E7F7FFFFFFFFFFFFFFF90
:10116000EFC0000000000000BCFEFFFFFFFFFFFF1C
:10117000FFFFFFFF3E3C000F1F7FFFFFFFFFFFFF52
:10118000FFEF010000007E3FFFFFFFFFFFFFFFFFBB
:10119000FFFFFFFF3F7E0000070F7FFFFFFFFFFF06
:1011A0007F3F0F0700003C3EFFFFFFFFFFFFFFFFF9
:1011B000FFFFFEBC000000000001EFFFFFFFFFFF8C
:1011C000FFFF7F1F0F001F1F0F7FFFFFFFFFFFFFAE
:1011D000FFFFFF3E000000000000C0EFFFFFFFFF29
:1011E000FFFFFF7F7F3E3F1FFFFFFFFFFFFFFFFF70
:1011F000FFFFFF7F0E0000000060FFFFFFFFFFFF0B
:10120000FFFFFFFCF87009080006060F0F1F1F3FC5
:10121000227F113F091F060F00060006060F0F1F51
:101220001F3F3E7F1F3F0F1F060F00060012127F59
:101230004FFF53FF1F7F53FF4EFF107E0010003EF5
:101240003E7F41FF55FF5DFF7FFF49FF77FF49FF6D
:101250007FFF41FF7FFF7DFF41FF7DFF3E7F003E1F
:101260000000003E3E7F7FFF41FF41FF41FF7FFFC7
:1012700041FF41FF41FF7FFF41FF41FF41FF7FFFF2
:101280003E7F003E000009080006060F0F1F1F3FAB
:10129000227F113F091F060F00060006060F0F1FD1
:1012A0001F3F3E7F1F3F0F1F060F00060012127FD9
:1012B0004FFF53FF1F7F53FF4EFF107E0010003E75
:1012C0003E7F41FF55FF5DFF7FFF49FF77FF49FFED
:1012D0007FFF41FF7FFF7DFF41FF7DFF3E7F003E9F
:1012E0000000003E3E7F7FFF41FF41FF41FF7FFF47
:1012F00041FF41FF41FF7FFF41FF41FF41FF7FFF72
:101300003E7F003E00000208020700073817150064
:10131000170A001202023E17130737001F020015BA
:10132000220A261E370D3800190D3E1C2414121EE9
:10133000300D070005152B00040302000A141D00E0
:101340002C1C001C2C0A181E1D0C320032063C00FE
:1013500003132100210A0002331C16001F03001290
:10136000270F0F001B12000603031C1E3A1B0C0064
:10137000031B3E0F320D00040E02021C23021F1E2F
:101380003B030B1E030C3C00230A130A021C3E1CE9
:101390002409240035161E1E1A0B3E1607183800A5
:1013A0000B173E1C0E1800123B020D1E11110200FD
:1013B0003C02301E3C1C1A001414230003050300D9
:1013C0003B1C2C1E090B000B321500063C1C0200B6
:1013D0003C020006120D251E0B02331E26160F00BE
:1013E0002F023E023619171E0B130007230A3E1266
:1013F0001B0721000602151E131300083B1C2300C7
:101400002412000321031C000303231E11073B00C9
:101410003816021E1804000E22141500150C191E91
:101420001C141B0033183E1C3B1C00033B023E02F5
:101430000305001C1802111E20190A000B140300DA
:101440002602001B02123E1C02023E041F081F1E41
:1014500021022B1E021C25001F1A0010230B39002D
:10146000021C1F1E0C0F3E122A0B1B001212000939
:101470002B0F2F1E151C3E1223193200040E3E1B8B
:101480001702001C1A0C3C1E231703002311131E05
:101490000C0D3E0C170A2B003C1C00072B1B1F00D9
:1014A0001406261E1F0F1A1E1F0C0C00021C3E1CC9
:1014B0001F0B0800021C3E1C0A022A1E19030A0008
:1014C00006193A002C1C3B003B02120002023E07A8
:1014D000190E3E1C241C1F003801120002023E0D92
:1014E0001F1800060C0F1B1E3A1B0C0024123E1284
:1014F0003B1C001332122B001C031F1E230200048E
:101500002E1533000E122C1E04033E0F181D040C62
:101510002F0B021C3A1C1F1903063C020C122D0C47
:10152000261010163204021C38192F0913173C021A
:1015300008101C0E370E06022C02021B12123B0F63
:1015400002092D0A0B171C143C0202022102021C84
:101550003B1B2A0A040A1F1214142E1B08053414FC
:101560002314100A3A02391B130A25033B02020A0C
:101570003802291C02022802171C3C1C2A0A0202FB
:101580001514241C3C023313230C021C0202120209
:1015900005021D1C33172602370F180A2C0A0205F4
:1015A00002122202021C1D0C3C1C02021307011D28
:1015B0002B133D140B172B071C1C321C1102081592
:1015C000320217123C120A02021C2A0A0B1C1F0FBD
:1015D0000B05140A3C122F0317130F03021C1303ED
:1015E000381B09143803270F031B300D1E04090292
:1015F0002A14180A021C2A130D1333073307191C67
:101600000A0A220A021C33171B1C0404180F2B079A
:101610000D0D241212023A04021C0E02021C3B1B86
:1016200014123C022A051B130F0E021C37150C0561
:1016300002123C1C220D1912340A2612021C1C0232
:1016400021053412130A360322030C16341000F855
:10165000FFFFFF7F0100000000F8FFFFFFDFCFCF9B
:101660004F0700FFFFFFFFFF00E0FEFFFF3F0F01FE
:10167000F8FFFFFFDFCFCF4F0700F8FFFFFF7F012D
:101680000000FEFFFFFFFFF0F0F01080FEFFFFFF05
:10169000F7F3F3F30000001FFFFFFFFFFFFF3F071B
:1016A000010080FEFFFFFFF7F3F3F30080FEFFFF72
:1016B000FFFFF0F0F0102208C0FFD9D9FF77007CBF
:1016C000FFC3E17F1F80FE0F3FF8FE1F007CFFC3BA
:1016D000C07C3F0160C6CFF97301CC2181219A21E2
:1016E00081216421812141232A08E0FE3FF0FF1F70
:1016F0000178FEC7C3E37F1E00F8FF19F9FF0780DA
:10170000FE3FFFF03CFFFF0780F83E27FFFF008011
:10171000F8FFC7C02E0880FE3FFFF03CFFFF0780A8
:10172000F83E27FFFF000083FF7C0F0300C0FEFF91
:101730001BF8FF0F0180FEFFD9D90180FE3FFFF0AB
:101740003CFFFF073608F0FF19191F0F00F8FF19BB
:10175000F9FF0780FEFFD9D90160C6CFF973016098
:10176000C6CFF973010000000080FE3F3CFFC301BB
:1017700080FEFFD9D9010083FF7C0F035410013F85
:10178000FFFFFFF0F0FEFF3F0F07C1F0FCFE3E1F22
:101790000F0FFFFEFEF880FFFFFF7F0100F8FFFF45
:1017A000FF3F010000000000FFFFFFFF03E0FCFF20
:1017B000FFFFFF00F0FFFF7F1FC3F0FCFE3E1F0F87
:1017C0000FFFFEFEF800F8FFFFFFFFFFF0C0FFFF76
:1017D000FF1F0000FFFFFFFF3F03000000001F7F0F
:1017E0007FFFF0F0F87C7F3F0F033F7FFFFFF0F0BB
:1017F000FE7F7F3F0700000000000000FFFFFFFFAB
:10180000FE3F0700FFFFFFFFFF1F0300001F7F7F5A
:10181000FFF0F0F87C7F3F0F83FEFFFF7F003FFF6C
:10182000FFFFFFFF070081218121812181210E22FD
:101830006A10C0F0FCFE7E1FCFCFDFCFC6C2000013
:1018400000E0F8FFFF1FFFFFFFF8000000F8FFFFB8
:10185000FFFFFFFE80E0FC7FFFFFFFFF1F0000F89F
:10186000FFFFFFDFCFCF4F070000000000C0F0FCFC
:10187000FE3E1F0F0FFFFEFEF800FFFFFFFFFF0001
:10188000E0FEFFFF3F0F01F8FFFFFFDFCFCF4F0765
:1018900000F8FFFFFFFF8F8FFFFFFE7C1F3F7FFFE2
:1018A000F8F2F3FFFF7F1F80E0FCFFFF3F1F1CFCEF
:1018B000FFFFFFFF0080FEFFFF7F01FFFFFF7F0FA5
:1018C000C3FFFFFFFF030080FEFFFFFFF7F3F3F30B
:1018D000000000000000001F7F7FFFF0F0F87C7F19
:1018E0003F0F03001FFFFFFFFFFFFF3F07010080C7
:1018F000FEFFFFFFF7F3F3F300C0FEFFFFFF070F4C
:10190000FFFFFFFDC0003A1000F0FFFFFFFF8F8FC9
:10191000FFFFFE7C0000E0F8FFFF1FFFFFFFF80065
:101920000080FFFFFF7F0100F8FFFFFF3F0100F88D
:10193000FEFEFFCF8F1F0F0602F8FFFFFFDFCFCFA6
:101940004F07FCFFFFFF1F070707070381E0FCFFAE
:10195000FF3F1F1CFCFFFFFFFF00003F7FFFFFF06A
:10196000F0FE7F7F3F074070F8F0F1F3FF7F7F1FAD
:101970000080FEFFFFFFF7F3F3F300000620C4949E
:1019800034044CF8FFFF00F80C07FF7F0003CEF88B
:10199000080A0B080C073E2000000000000000F8B9
:1019A0004C043494C4E4E4E46424AC28282C2424B7
:1019B00064E4E4ECECE4242CE8E8E82828E82828AF
:1019C000EC242424242C7CEC2424E4E42424E46467
:1019D0002C2CE42464EC000000000080C0474CD0B4
:1019E000803FFFFF87B338B9D9410000183838B3BA
:1019F00087FFFFFFF8E0838F83E0F8FF8080FF819F
:101A000081E3C1889CFFC0809F9F80C0FFCC88F885
:101A10008382C6FFF0F8C09EBFBF3C3898CC073029
:101A200071C0C04372604C5E525E4C607243404075
:101A3000F1FF80809F9FFFC1C08E80A0FF8080F655
:101A4000F0F0FFF3F3FEFE8E82F0F8FFB0B6B68042
:101A500080FF0001010101000000030604040404EA
:101A6000003E7F411C3E7F7F7F7F6341633E0004D9
:101A70000C08080C0C0808181018080808080808B2
:101A800008080808080808080808080808080808D6
:101A90000B0B0B0B0B0B0B0B0B06060606060606B9
:101AA0000B000000000000000B000000010000001F
:101AB0000B000100000001000B000000010000000D
:101AC0000B000100000004000B00000001000000FA
:101AD0000B0B0B0B0B0B0B0B06060606060606067E
:101AE00000000000000000000300000001000000F2
:101AF00000000100000001000100000001000000E2
:101B000000000100000001000100000003000000CF
:101B10000B0B0B0B0B0B0B0B060606060606060B38
:101B2000000000000000000B010000000100000B9D
:101B3000000004000000000B010000000100000B89
:101B4000000001000000000B010000000100000B7C
:101B50000B000100000001000B000000010000006C
:101B60000B000100000001000B000000030000005A
:101B70000B000100000001000B000000010000004C
:101B80000B000100000001000B000000010000003C
:101B90000000010000000100010000000100000041
:101BA0000000010000000100010000000100000031
:101BB0000000010000000100010000000100000021
:101BC000000003000000010001000000010000000F
:101BD000000001000000000B010000000100000BEC
:101BE000000001000004000B010000000100000BD8
:101BF000000001000000000B030000000100000BCA
:101C0000000001000000000B010000000100000BBB
:101C10000B000100000001000B00000001000000AB
:101C20000B000100000001000B0000000400000098
:101C30000B000100000001000B000000010000008B
:101C40000B000000000000000B0B0B0B0B0B0B0B31
:101C50000000010000000100010000000100000080
:101C6000000001000000030001000000010000006E
:101C70000000010000000100010000000100000060
:101C800000000000000000000B0B0B0B0B0B0B0BFC
:101C9000000001000000000B010000000100000B2B
:101CA000000001000000000B010000000100000B1B
:101CB000000001000000000B010000000100000B0B
:101CC000000000000000000B0B0B0B0B0B0B0B0BB1
:101CD0000000010000000100010000000100000000
:101CE00000000C0E1216010001000D0F131700006A
:101CF0000000011014000100010000111500000097
:101D000000000100000003000100000001000000CD
:101D1000020202020202020202181A0202181A0247
:101D200002191B0202191B02020202020202020233
:101D3000020202020502020202181A0202181A0224
:101D400002191B0202191B02020202020202020213
:101D50000B0B0B0B0B0B0B0B0606060606060606FB
:101D60000202020202020202020202020202020253
:101D7000020202020202020202181A0202181A02E7
:101D800002191B0202191B020202020202020202D3
:101D9000020202020202020202181A0202181A02C7
:101DA00002191B0202191B020203020202030202B1
:101DB0000202020202020202020202020202020203
:101DC00002020202020202020B0B0B0B0B0B0B0BAB
:101DD00002020202020202020102030202020402E1
:101DE00002020202020202020202020202020202D3
:101DF00002020202020202030205020202020202BF
:101E000002020202040202020202020202020202B0
:101E1000000001000000000B010000000100000BA9
:101E200000000C0E1216000B01000D0F1317000B13
:101E3000000001101400000B010000111500000B40
:101E4000000001000000000B010000000100000B79
:101E50000B0B0B0B0B0B0B0B062625252525240640
:101E600000272727232323000127272723232300B5
:101E70000020212121212200011C1D1E1F1E1F00E8
:101E8000000708090A090A0001000000010000001B
:101E900001111112395F4FF539544445678777783E
:101EA0000111111235FF399E024701456777777896
:101EB0000111111235FF4FFE0244404E67777778CB
:101EC0000BBB11123DAD0F253DAA64856CCC777814
:101ED0000F1BB1F2393DD595390BB295677CC778A8
:101EE000011111123D3F02DE3A673EDE6CCC77787D
:101EF0000F1211F23494449E01149112677877788E
:101F0000011111123F2440F5348BB645677777787D
:101F1000011111123F14242539468485677777789B
:101F200001111112301FF19539777785677777782E
:101F300002F2F2F2344E444E3E444E4568787878D0
:101F40000011111231F3F0F53673467E677776781B
:101F50000011111233F68F253677788567777778F9
:101F60000F0F0F1234343445313442AE677768C8EE
:101F70000111111268F1F29E3447789E67777778E5
:101F80000F0F0F023737373E3949494E6777777859
:101F90000BBBBBF23AA99ADE3AA99ADE6CCCCCC84C
:101FA00002121BF233555AA53EE9EA0568787C68AF
:101FB00000111102333E111534FF40926677767896
:101FC0000B0112F23129904E341991456C6778C893
:101FD0000FFFFFF2344444453FFF9FF26777777865
:101FE00001111112399999953999999567777778EF
:101FF000011111F23E4443953EBB30F267CC677845
:10200000011111B233F1F2A530F1F2A5667777C86C
:10201000011111B2301902A5330925F267877778CB
:102020000BBFBBB23AADAAA53AADAAA56CCCCCC841
:102030000F0F11123439ED3531012D0267767778A3
:1020400001F111123344999531131F156776778882
:10205000011BB01239EAAF9E39EAAD9E677CC778A2
:1020600002BB2F1231DD04E5042121256878787840
:10207000011211123111112531F11F15677877788E
:1020800000F10B0233B3BD2536B3F32E67777678B4
:102090000810E0FC3E0F070FFFFE3F7FF8F0F0F85E
:1020A0007F1F00001CFEFFFF00000000E0FFFF7F1D
:1020B0006000001C1E0783C7FF7EF0FCEEE7E361B3
:1020C0007070000E0F87C3E7BF1E70F8F8F0E0F1E4
:1020D0007F3FC0F0FC8F83FFFEC003030303FFFFBD
:1020E0007F0000FEFEC7C7C7C78378F8F0E0E0F1C5
:1020F0007F3FE0F8BCCEC7C380003F7FF1E0E0F156
:102100007F3F0E0F0F07C7F37F0F0000F0FE1F0386
:102110000000007CFEE7C3E77F3E3E7FF3E1E1F392
:102120007F3EFCFE8F07078FFEFC0001C3E3733D7B
:102130001F070808007C7CFEFEFFC7FFE3FF7FFF50
:102140003E7F003E0000000606CFC6FFFFFFFFFFF8
:1021500007FF000700C0C0E6E6FFF7FFFBFFDFFF59
:102160000EDF000E0000004242E7E7FFDBFFFFFF4B
:102170007EFF007E006060F878FE7EFFE7FFFFFFD5
:1021800067FF00670000005050FFDFFFDFFFFBFF2D
:1021900073FF0073007070F8F8FECEFFCFFF7FFF73
:1021A00079FF0079008080C3C3F7F3FF7FFF1F7FB3
:1021B000071F0007007070FFFEFFDFFFCBFFFFFF70
:1021C0007EFF007E0000009E9EFFDFFFF3FF3FFFCB
:1021D0001E3F001E0308000E000D000F020A080E2D
:1021E0000A00181B00080A02000A021E1E00000A4C
:1021F00000080A0025203E3C1C0C0683C1E1F1F1D9
:10220000F1F1F1E1C3860E1E3C70F0F0F0F0F0E069
:102210000000000000000000000000FE83001E3FE0
:102220007FFFFFC18C06064E7C3983FF7E7C68C031
:10223000810347CF9C3C78C0800000000000000074
:10224000C06123060C1830612367EF4F0F1F3F71E9
:1022500020081C3EFCF9F0F0FCFEFCF8F0E143869F
:102260000C38F00000060C183060C080000000023E
:10227000060C1803063C78F2E7CF9FBFBF9FCF67DD
:1022800033190C0683E0387FC0803E40FFFFFFFF1C
:10229000FFFFFFFFFFFFFFFFFFFFFFFFFFFFFFFF4E
:1022A0007F3FFFFFFFFF7F3F9FC7FFFFFFFFFFFF56
:1022B000FFFFFFFFFFFFFFFFFFFFFFFFFFFFFFFF2E
:1022C00000FFFFFFFFFFFF0000FFFFFFFFFFFFFF1B
:1022D000FFFFFF7F7F7F7F7F7F6FE763613486F340
:1022E000FB791DFCFEFFFFFF3F8FFFFFFFFFFF3F5E
:1022F00080C71FFFFFFFFFFFFFFFFFFF1FC3F8FFA8
:10230000FFFFFF1F01C07C073FFFFFFFFF7F1F0391
:10231000F8FEF77359198BC2C6FCF03A8BE1F8FC52
:10232000FFFF3F8FE3F0FCF9FBF3E7E370707363AB
:10233000604FCF8F8F2FEFE70398FE7F3F9FCF63D4
:1023400030180E03000000818791FCFEF0F8F9F3CD
:10235000E7EECCDCD90F87E3F87E3F9FCFE7F3F8B9
:10236000FEFFCF8F0F1F1F3D3C3878787CEFE6F0E3
:10237000FCFFFFFF8338ECC4C6C2C3C180808080ED
:1023800000000000F8E38F3FFFFFFFFF7F7F3F0F5C
:1023900087C1CC0673F9FCFEFFFFFFFFFFFFFFFFC5
:1023A000FFFFFFFFFEFEFCFCFCFCFCFFFFFFFFFF4E
:1023B0007F7F3F9ECCE1F3FFFFFF7F3FBFBFBFBFEB
:1023C000BFBEFFFFFFFEF8F3E7CF9E3E7F3F1F0F2C
:1023D0000F07040133E7CF9F3F7FFFFFFFFFFFFFA2
:1023E000FFFFFFFF7F7F7F773783E3F3F3F9FCFF86
:1023F000FFFFFFFFFFFFFFE04C1D1D0D05010180EA
:10240000F9F3F7EFCFDFBFBF3F7F7EFCFCF8F8F8B2
:10241000F8F8FCFF7F1FC7D0DEDC9DB9BB3B7B79A2
:10242000FDFCFEFFFFFFFFFFFFFFFFFFFFFF7F3F02
:102430001F0F070381C0C06030386CC68381FFFF67
:10244000FFFFFFFFFFFFFFFFFFFFFFFFFFFFFFFF9C
:10245000FFFEFEFFFFFFFFFFFFFFFFFFFFFEFEFC93
:10246000FDF9F3F77F3F1F0F07030180C070381895
:102470000C07030100000000000001033C380000CD
:1024800000000080F8FE0FE3FB1B0B0B8BFBF3F748
:10249000F6F6F60606ECECECECECECECECECECEC2A
:1024A000ECECECEEE6F6F6F6F7F3FBFBCBCBFBE35E
:1024B0000FFEF8801E332121339E00000080F8FFBC
:1024C0000FE0F8F9F9F9F9F9F9F9F1F3F3F3F3F0A9
:1024D000F0FFFFFFFFFFFFFFFFFFFFFFFFFFFFFF1B
:1024E000FFFFFFFFFFFFFFFFFFFF7F7FFEE00FFF0C
:1024F000F880060600000000000F3FF0C607040445
:10250000070707070707070707070707FFFFFFFF7B
:10251000FFFFFFFFFFFFFFFFFFFFFFFF07070707AB
:1025200007078787070726860707C6F03F1F008033
:102530008000000000000000030784C4E4E4E4E439
:10254000E4E4E4E4C49C000FE7E7E7E7E7E7E7E754
:10255000E7E7C7870F1F0FC7E7E0ECE4E4E4E5E532
:10256000E4C4040404070300C040C30311000000D6
:10257000000000000000FFFFFFFFFF393939FFFFB7
:10258000FF0FE0E0EFEF0FFFFF183879FFFFF703D1
:10259000E0E0EFEF0FFFF9F0F0FCFDFDFD0DECE0EA
:1025A000E0E00000012101000000000080C0602088
:1025B00060C080000000000C0C007EFE803C3E1CD1
:1025C0001C1C1C1C0C0C0E0C0C0C0C0E1E1C1C1CC5
:1025D0001C3C3E80FE7E00000000C0E0E0C0000029
:1025E0000000030300000E1B3166C680D060311B63
:1025F0000E00003828380001471E382020202030E7
:102600001010D0D0101090103020202020381E073D
:1026100001000006060000010100000000000000AB
:1026200000004020FFFFFF0707E7E767676767676E
:1026300067E7E70707FFFF9F9FFFFF8787FFFF67AA
:1026400067E7E7FFFF9F9F67679F9FE7E76767E78A
:10265000E7FFFF0707E7E7676767676767E7E7077A
:1026600007FFFFFFFFFFFF00007F7F60606060608B
:10267000607F7F0000FFFF1919818179799F9F1882
:1026800018F9F901019F9F7E7E81816161E6E60173
:1026900001FFFF00007F7F6060606060607F7F00FF
:1026A00000FFFFFFFFFFFFE6E6E6E6E6E60606863A
:1026B000867E7E666687878686E1E11818E1E19E60
:1026C0009E87876666797918186767FEFE8181980C
:1026D0009887879E9E86861E1EE6E6FEFEE6E69E9E
:1026E0009EFFFFFFFFFFFF9999191901018080FFED
:1026F000FF98986666E7E7E7E7676766667F7F614A
:10270000618787606060601E1E86869999818179E5
:10271000791F1F9F9F81819898E7E70707F9F99F25
:102720009FFFFFFFFFFFFF1919808086861919E1BF
:10273000E1E7E766660707F9F918181E1EE0E09E54
:102740009E1F1F7E7E60608080E7E7797999999867
:10275000989E9E1F1F79799F9F1F1F0606F9F99F5C
:102760009FFFFFFFFFFFFF60607F7F616166666123
:102770006167676666E0E001011E1E86867F7F61F5
:1027800061F8F8E6E67E7E1919E7E77E7E191907FB
:1027900007E7E76666E0E001011E1E060681818705
:1027A00087FFFFFFFFFFFF0000FEFE06060606068E
:1027B00006FEFE0000FFFF060686861F1FE0E09E65
:1027C0009E1F1F191960601E1E878780809898E0E1
:1027D000E00707666607076060000066660101871C
:1027E00087FFFFFFFFFFFFE0E0E7E7E6E6E6E6E65C
:1027F000E6E7E7E0E0FFFFE0E0FFFFE0E0FFFFE10A
:10280000E1F8F8E6E6F8F8F8F8E7E7FFFFE7E7F9B8
:10281000F9FEFEF8F8E0E0E6E6E0E0E6E6F8F8FFCC
:10282000FFFFFFFF0620C49434044CF8FFFF00F8BC
:102830000C07FF7F0003CEF8080A0B080C073E20A8
:1028400000000000000000F84C043494C4E4E4E408
:102850006424AC28282C242464E4E4ECECE4242C48
:10286000E8E8E82828E82828EC242424242C7CEC18
:102870002424E4E42424E4642C2CE42464EC000008
:1028800000000080C0474CD0803FFFFF87B338B9BD
:10289000D9410000183838B387FFFFFFF8E0838F75
:1028A00083E0F8FF8080FF8181E3C1889CFFC080C6
:1028B0009F9F80C0FFCC88F88382C6FFF0F8C09E3F
:1028C000BFBF3C3898CC073071C0C04372604C5ECB
:1028D000525E4C6072434040F1FF80809F9FFFC179
:1028E000C08E80A0FF8080F6F0F0FFF3F3FEFE8E36
:1028F00082F0F8FFB0B6B68080FF00010101010050
:102900000000030604040404003E7F411C3E7F7F58
:102910007F7F6341633E00040C08080C0C08081814
:10292000101808080808080808080808080808080F
:10293000080808080808080810081F09091F001FD0
:102940000909170001011F01000A15081F111111C3
:10295000001F11111F001F11110E001F151511006E
:102960000A39208E5951D78600001F0505C100DFA6
:102970005050DF005F51D11FC05F45C50740C744BD
:102980001C070000002020F8202000000000B8A84C
:10299000A8E8000808F80800F888A8E8834644C5B5
:1029A000810000C244444700C74444C700C54547AE
:1029B00040074242C54004C74440C00040C04000F8
:1029C000C00000C000C040404000C0000000000047
:1029D0000000000000E3961475610000870404F411
:1029E00000F70202F700755555D7001010F71010C8
:1029F0000711F11100F4274480F6010106000705D4
:102A0000F5141017047444C07000F090907038658D
:102A1000455D1800002041417D007D45457D005504
:102A2000557D017C24245D00447C450101000100AA
:102A3000000001000101010100010101010000008D
:102A4000010000010000011D08FF81BD8989BD81D1
:102A5000BDADADA581BDA1AF81BD95D5DDC1FFFFE8
:102A6000FFFFFFFFFFFFFF81BD95D5DD81BDA1AF5A
:102A700081BD9595BD81DD91B19DC1FFFFFFFFFF38
:102A8000FFFFFFFF81A5BDA581BD8991BD81BD95DA
:102A900095C581BDA5A5BD81FFFFFFFFFFFFFFFF1E
:102AA000FF81BDA5A5A581BDA5A5BD81BD8991BDA0
:102AB00081BD95D5C1FFFFFFFFFFFFFFFFFF81AD88
:102AC000ADADB581BD959581A59989A581FFFFFF24
:102AD000FFFFFFFFFFFFFFFFFFFFFF81BDA5A5BDBC
:102AE00081BD959581BD959581FFFFFFFFFFFFFF9C
:102AF000FFFFFFFFFFFFFFFF81BDA5A5BD81BD89D2
:102B000091BD81FFFFFFFFFFFFFFFFFFFFFFFFFF03
:102B1000FFFFFFFFFF81BD8991BD81BDADADA581E7
:102B20009DB199B19D81FFFFFFFFFFFFFFFFFFFFF9
:102B3000FFFF81BDA5A5A581BDA5A5BD81BD8991CD
:102B4000BD8185BD85F1FFFFFFFFFFFFFFFFFF8117
:102B5000BD8989BD81BDADADA581BDA1AF81BDA13F
:102B6000AF8FFFFFFFFFFFFFFFFFFF010204081011
:102B7000204080D5F08D14A1C881CFD9F1AF2000BD
:102B80005810F0F89C8E8783878E9CF8F00000FE2A
:102B9000FF0303030303070EFCF80000FEFF03031B
:102BA000030303070EFCF80000FFFF000000000015
:102BB0000000FFFF0000FEFF8383838383C7EE7C5A
:102BC000380000F8FC0E07030303070EFCF80000B2
:102BD0003F7FE0C08080C0E07F3FFFFF0101010137
:102BE000010101FFFF0000FFFF0C0C0C0C1C3E77E5
:102BF000E3C100007FFFC0C0C0C0C0E0703F1F0045
:102C0000001F3F70E0C0C0C0E0703F1F00007FFFAA
:102C1000C1C1C1C1C1E3773E1C00001F3F70E0C0CD
:102C2000C0C0E0703F1F000000000001FFFF010076
:102C30000000462241252B22A7248B2A022AED22BE
:102C40003A27DA16FD265E22D42640218B22202147
:102C500008080000000000000000080B000202024B
:102C60000100090400000102020000052400100117
:102C700005240101010424020605240600010705BC
:102C8000810310004009040100020A00000007054A
:102C9000020240000007058302400000040309040B
:102CA00012010002EF0201404123368000010102BF
:102CB000030141726475696E6F204C4C4300417290
:102CC0006475626F7900D83411241FBECFEFDAE04B
:102CD000DEBFCDBF11E0A0E0B1E0E6E7FDE602C057
:102CE00005900D92A834B107D9F727E0A8E4B1E028
:102CF00001C01D92A636B207E1F716E1C4E6D6E19F
:102D000004C02197FE010E94AE36C336D107C9F731
:102D10000E9441330C94B9360C940000EF92FF925C
:102D20000F931F93CF93DF931F92CDB7DEB77C0134
:102D3000FC0100811181C80169830E940D366981FF
:102D4000681719F0C8010E941536C7010F90DF916E
:102D5000CF911F910F91FF90EF9008950F93DC0199
:102D600017968C911797882311F1ED91FC9111978B
:102D7000CB01820F911D27FD9A95E817F907BCF446
:102D80003F96E617F7079CF012968D919C9113974A
:102D90009A01200F311D07FD3A95821793073CF4E5
:102DA0009C01215F3F4F81E0241735070CF480E040
:102DB0000F9108952F923F924F925F926F927F9260
:102DC0008F929F92AF92BF92CF92DF92EF92FF923B
:102DD0000F931F93CF93DF93CDB7DEB769970FB6ED
:102DE000F894DEBF0FBECDBF809106018E3011F486
:102DF0006FE001C06CE3862F880F680F70E0809150
:102E0000E7069091E8060E9486368C01892B09F02E
:102E100071C00E94993520ED31E040E050E00E9401
:102E200023366B017C0120E1C20ED11CE11CF11C98
:102E30000E94993520ED30E040E050E00E942336BA
:102E40002B013C0130E1430E511C611C711C80912F
:102E5000D2029091D302AC0140585109C416D50654
:102E60007CF080589F4F8C159D0554F08091D402C2
:102E70009091D502AC0140545109441655061CF4FA
:102E8000E4EEF1E00CC0805C9F4F84159505C4F31F
:102E900031C00F5F1F4F3A960831110559F18081FB
:102EA0008111F7CF0E94993523E030E040E050E0F7
:102EB0000E9423368AE0809FF001819FF00D11244B
:102EC000E352FE4F148281E087831582D182C08253
:102ED000538242826187662311F082E001C083E061
:102EE00086838AE0809FF001819FF00D1124E352D8
:102EF000FE4F10860E94C72A8C708C3019F48AE02D
:102F00008093CD028091DC02843218F081E08093BE
:102F1000DB021A8219821091CF020E94C72AEE2486
:102F2000E39485FFE12C0E94C72A5524539486FF21
:102F3000512C0E94C72A082F001F0027001F0E9443
:102F4000C72AFF24F39484FFF12C0E94C72A44244B
:102F5000439483FF412C0E94C72A51E05B8382FF88
:102F60001B82011106C0F11006C0EE2031F08E2D3B
:102F700005C0802F03C08F2D01C0852D8093CE0208
:102F80008091D902882319F081508093D9020111D0
:102F900002C0FF2021F0E1106AC2511068C2809186
:102FA000D102882319F081508093D102EE2011F0D4
:102FB0008FEF03C0552011F081E08A832A81809130
:102FC000D2029091D302820F911D27FD9A95909382
:102FD000D3028093D2029E012E5F3F4F41E064ED09
:102FE00072E082ED92E00E94122E9E012E5F3F4F12
:102FF00041E064ED72E082ED92E00E94702E0023C9
:1030000011F08FEF03C0FF2011F081E08983298147
:103010008091D4029091D502820F911D27FD9A953F
:103020009093D5028093D4029E012F5F3F4F40E0E2
:1030300064ED72E082ED92E00E94122E9E012F5FFD
:103040003F4F40E064ED72E082ED92E00E94702E0E
:103050008090D4029090D5026090D2027090D302FA
:1030600094E9A92E91E0B92E20E9222E21E0322EFA
:103070006101A301405F5F4F9401205F3F4F71E00A
:10308000D5018C918823B1F1F6018081918184175B
:10309000950784F50F968615970564F182819381D3
:1030A000821793073CF50F96881599051CF1F501D9
:1030B000108284E992E0288F398F4D8B5E8B7F8B55
:1030C0000E94B82B8091A9019091AA018C509E4F2B
:1030D0009093AA018093A90180E090E0288D398D1A
:1030E0004D895E897F89FC01E057FE4F648166232C
:1030F00009F49EC1F5E0AF0EB11C85E0C80ED11CED
:1031000099EAC91691E0D90609F0BACF8091B501C4
:10311000A090D202B090D3028090D4029090D502B9
:103120008823E9F08091B1019091B2019501215F6E
:103130003F4F281739079CF00F968A159B057CF0A6
:103140008091B3019091B4019401215F3F4F281702
:1031500039072CF00F96881599050CF071C18BE793
:10316000682E81E0782EA7E7B1E0BE83AD836D01C4
:103170009501215F3F4F3C872B87A401415F5F4F43
:1031800058874F83D3012C91222389F1F601808146
:1031900091814B855C85481759074CF10F968A152C
:1031A0009B052CF1828193814F81588548175907DF
:1031B000F4F00F9688159905D4F0223041F484E993
:1031C00092E00E94B82B82E00E94F22D0EC080E7B0
:1031D00093E00E94B82B8091A9019091AA018C598B
:1031E0009F4F9093AA018093A901D3011C92B8E04C
:1031F0006B0E711CE8E0CE0ED11CFFE8CF16F1E09B
:10320000DF0609F0BFCF41101FC0EE2031F00111E1
:1032100012C0FF2091F011E017C0552031F00111CC
:103220000EC0FF2071F017E00FC001110CC0FF208D
:1032300059F010E009C013E007C012E005C015E026
:1032400003C016E001C014E01093CF025B81552348
:1032500011F0442009F010FF1093D8028091E70686
:103260009091E80683709927892BF1F48091DC0214
:10327000823018F081508093DC020E94C72A83FFBD
:1032800005C08091DB02811105C0DEC00E94C72A03
:1032900082FDF7CF8091DB02882389F09091DA02DA
:1032A00081E089278093DA025B81552329F08091A0
:1032B000DB02811144C007C04110F9CF40C05B81DF
:1032C000552309F4D8C08091D102811138C02091D2
:1032D000D4023091D5024091D2025091D302809114
:1032E000CF0290E0FC013696E770FF27E85EFE4FC4
:1032F0006081FC01E85EFE4F7081EFE4F1E080E068
:1033000090E0A081A111A6C0A7E0A89FF001A99F0D
:10331000F00D1124E75BFE4F475F5F4F5183408301
:10332000255F3F4F338322837483658381E08683E7
:1033300088EB91E00E94B82B8AE08093D1028091C3
:10334000DB02882349F08091DC02823028F410925D
:10335000DB0281E08093DA028091E7069091E80633
:1033600066E070E00E948636892B21F48091CE02BF
:10337000811177C08091D002843010F01092D00279
:103380008091A9019091AA0118161906C4F4059715
:103390009093AA018093A9018091AD019091AE0113
:1033A000A091AF01B091B0010596A11DB11D809310
:1033B000AD019093AE01A093AF01B093B0018091A5
:1033C000D702882319F081508093D7028091D802C8
:1033D00090E0FC01E85EFE4F2081A091D202B09106
:1033E000D302D897E4E02E02A00DB11D1124FC01F8
:1033F0003696E770FF27E85EFE4F80816091D40229
:103400007091D5026C517109F4E08F02600D711D4D
:1034100011242091730130917401A217B30774F144
:1034200041E02A173B070CF040E0CD01D90128C04C
:1034300005968931910509F056CE7093B5015ACEA3
:1034400086E08093CD028BCE8091DC028E5F8093EC
:10345000DC0220CF019637968630910509F051CFD6
:103460006BCF8091D0028F5F8093D00283CF84E0B6
:103470008093D90294CD411026CF61CFC9014FEF7F
:10348000042E000C550B8A1B9B0BFC01EE0FFF1F3B
:103490008E0F9F1F97FD0F96F4E095958795FA95EF
:1034A000E1F70196489FF001499FF00D589FF00DFC
:1034B0001124E20FF31F20917501309176016217FC
:1034C000730744F041E0261737070CF040E0CB01CA
:1034D000B90102C0C9014FEFF7FF02C0E0E0F0E020
:1034E000E138A1E0FA0714F0E0E8F1E0F0937401AC
:1034F000E0937301042E000C550B861B970BBC0147
:10350000660F771F860F971F97FD0F9664E09595BE
:1035100087956A95E1F70196489FB001499F700D24
:10352000589F700D1124260F371F37FF02C020E06F
:1035300030E0213C310514F020EC30E0309376018E
:10354000209375018FE4C82E81E0D82EE9E4F1E0E4
:10355000FC87EB877F0115E0D6018C91882309F465
:10356000DCC0F60132978081F70140805180480E1F
:10357000511C87FD5A9451824082F6013197808117
:10358000D70112968D909C901397880E911C87FD01
:103590009A9413969C928E921297BDED6B2EB1E089
:1035A0007B2EA12CB12C02E022E0A401B201C301C8
:1035B0000E94AE16882309F468C0F6011082FAE072
:1035C000FA9DC001FB9D900D11249C0123523E4F9A
:1035D0005901D90116968C911697815016968C93A5
:1035E00081114BC08CED90E00E94B82BF501108743
:1035F00017828091A9019091AA018C599F4F9093B5
:10360000AA018093A9018281938120813181409117
:103610007B01442359F040918301442351F04091B0
:103620008B0141113DC0E2E0F0E005C0E0E0F0E0D8
:1036300002C0E1E0F0E0A3E0EE0FFF1FAA95E1F782
:10364000E958FE4F41E0478316822C5F3F4F31839C
:10365000208304969383828380918F01A82FB0E00A
:10366000A05EBE4F9C9194838F5F8A3018F4809344
:103670008F0116C010928F0113C0D90118961C93A8
:1036800080E892E00E94B82B0BC0BFEFAB1ABB0AD8
:10369000EAE06E0E711CF8E1AF16B10409F083CFB9
:1036A000D70112966D917C91139777FF02C0695FE5
:1036B0007F4FF3E075956795FA95E1F7F701808103
:1036C000918197FD0796E3E095958795EA95E1F757
:1036D0000E9499278B3010F0D6011C92F70160816F
:1036E00071812091730130917401621773079CF00E
:1036F0004281538180917501909176014817590755
:1037000054F020583F4F261737072CF0805C9F4F0E
:103710008417950714F4D6011C92B7E0CB0ED11C88
:10372000E7E0EE0EF11CF3E7EF16F1E0FF0609F01B
:1037300013CF24EEC22E21E0D22E2DED31E03C83BA
:103740002B8341EEA42E41E0B42E790153E0452EA7
:10375000512CD6018C91882309F4E4C01A82198275
:103760008091E7069091E806B2010E948636892B87
:1037700009F0D1C0F701808191812091D20230916E
:10378000D3028217930714F421E004C028173907E5
:1037900014F42FEF2A83D70112962D913C911397A1
:1037A0004091D4025091D5022417350714F441E01A
:1037B00004C04217530714F44FEF49838115B2E058
:1037C0009B0708F0ADC02F3F310511F008F0A8C0ED
:1037D0002A8127FF04C0F6013297108206C02223F7
:1037E00021F031E0F60132973083820F911D27FDE1
:1037F0009A95D7018D939D933D019E012E5F3F4F7A
:1038000041E0BD01C7010E94122E8090D20290902B
:10381000D3024091D4025091D50200E120E1B401DD
:10382000C7010E94AE168823B1F08A8118163CF4B5
:10383000B0E18B1A9108F7019182808208C0882339
:1038400031F0F0E18F0E911CD7018D929C928FEF99
:103850000E94F22D1A829E012E5F3F4F41E0B3017C
:10386000C7010E94702E2981F70182819381820F06
:10387000911D27FD9A95938382839E012F5F3F4F71
:1038800040E0B301C7010E94122E8090D4029090B4
:10389000D5026091D2027091D30200E120E1A4012F
:1038A000C7010E94AE168823C1F0898118164CF416
:1038B000F0E18F1A9108D70113969C928E9212977D
:1038C00008C0882331F0B0E18B0E911CF701938280
:1038D00082828FEF0E94F22D19829E012F5F3F4F4F
:1038E00040E0B301C7010E94702E8A81811103C09C
:1038F0008981882371F08091E70680FD04C0D5019D
:103900008C918F5F8C93F5018081883020F010823C
:1039100002C0D5011C92F60131978081811102C04D
:10392000F6011082FAE0CF0ED11C2AE0E20EF11C63
:103930003AE0A30EB11C4DECE41642E0F40609F0A7
:1039400008CF8091E7069091E8066AE070E00E9457
:103950008636892B29F4809148018F5F8093480136
:1039600080914801843010F010924801E090750178
:10397000F09076010091730110917401C801F3E099
:1039800096958795FA95E1F798878F83680197E078
:10399000C922DD24D70183E0B695A7958A95E1F782
:1039A000BE87AD875701B7E0AB22BB24712C98E2EC
:1039B000692E872D90E0C114D10419F420E130E084
:1039C00002C021E130E0821793070CF047C063E0AA
:1039D000880F991F6A95E1F7FC01EC19FD09F88B36
:1039E000EF87512C8F809884870C911C252D30E017
:1039F000A114B10419F488E090E002C089E090E0DD
:103A0000281739074CF56D857E85620F731FC40139
:103A1000288F398F0E949927482F8091AB01909170
:103A2000AC01019763E070E00E949A36689E400DF9
:103A30001124288D398DB901E3E0660F771FEA95CF
:103A4000E1F76A197B09242F4CEA50E08F859889A9
:103A50000E94FC295394CACF7394ABCF8091B501D7
:103A6000882309F481C08091B801811107C0809139
:103A7000B901882319F081508093B9018091B9016F
:103A8000811106C08FEF0E94F22D8FEF8093B90154
:103A90008091E7069091E8066AE070E00E94863621
:103AA000892B61F48091B7018F5F8093B70180917A
:103AB000B801882319F081508093B8018091B80132
:103AC000813019F48FEF0E94F22D8091B70184307C
:103AD00010F01092B701E12CF12C00E010E0A09062
:103AE0007501B0907601C0907301D090740160911F
:103AF000B3017091B4016A197B09600F711F809145
:103B0000B1019091B2018C199D0920E044E955E082
:103B10008E0D9F1D0E94C12A2091B601220F220FF7
:103B20008091B701280F6091B3017091B4016A19B7
:103B30007B09600F711F8091B1019091B2018C19C6
:103B40009D0942E155E08E0D9F1D0E94FC29085FF2
:103B50001F4F0031110519F6F8E0EF0EF11C20E1BE
:103B6000E216F10421F1B9CF6091B3017091B40173
:103B70006E197F098091B1019091B20120E040EF70
:103B800054E0801B910B0E94C12A6091B301709197
:103B9000B4016E197F098091B1019091B201209119
:103BA000B6014EE654E0801B910B0E94FC293EE7D3
:103BB000C32E31E0D32E0CE711E04DE7E42E41E0B7
:103BC000F42E56E0A52EB12C992493942091E7066B
:103BD0009091E806822FB5010E948636892B41F428
:103BE000D7019C919F5F9C93F80190819F5F908388
:103BF00020FD05C0D7018C918A3108F003C3F7017D
:103C00008081F80131978F3108F01082D8018C91B2
:103C1000863008F01C928081882319F1F60190818A
:103C20009923F9F090E00197282F220F820F880F37
:103C3000D8012C91280FED81FE81628173818091E2
:103C4000750190917601681B790B80819181E091DB
:103C50007301F09174014EE955E08E1B9F0B0E9499
:103C6000F629F8E0CF0ED11C2D813E81285F3F4F11
:103C70003E832D83085F1F4F38E0E30EF11C4D811A
:103C80005E814F58514009F0A1CF8091E706909195
:103C9000E8066EE170E00E948636892B31F490913F
:103CA000000181E089278093000101E011E025E017
:103CB000B22EB00ED10114968C911497882309F47A
:103CC00043C0C0907501D0907601E0907301F090F0
:103CD000740112966D917C9113976C197D098D91E9
:103CE0009C91F801208144E559E08E199F090E94BA
:103CF000C12AD8012C91220F220F80914801280F50
:103D0000F101628173816C197D098081918142ED9D
:103D100056E08E199F090E94FC298091000188239A
:103D200099F0D10112966D917C91139769507109A8
:103D30006C197D098D919C91409620E040E656E0FB
:103D40008E199F090E94F629B5E02B0E311C0F5FDA
:103D50001F4FB012AFCFE2EEF1E0FE83ED8395EEA0
:103D6000492E91E0592EF20131979081D2018C9128
:103D7000992309F452C0882311F081508C93F201E9
:103D800080818370823008F02FC1AB81BC810D919E
:103D90001C9111978091730190917401081B190B6C
:103DA0001296ED90FC901397809175019091760199
:103DB000E81AF90A19968C9134976F018823A9F0B3
:103DC000AD81BE812C914CEB5CE0B701C8010E9433
:103DD000C12AED81FE818081D6012C91B8E08B9FB4
:103DE000200D11244AEB5AE013C0ED81FE812081A1
:103DF00048E75AE0B701C8010E94C12AD6012C91B8
:103E00002170ED81FE818081880F280F46EF59E0F7
:103E1000B701C8010E94FC29E7C0882309F4E4C067
:103E20008150D2018C93EB81FC8182809380209120
:103E3000750130917601821A930A7401F8E0EF0E51
:103E4000F11CAB81BC81AD90BC902091730130918D
:103E50007401A21AB30A6501B8E0CB0ED11C06E0CA
:103E600010E0081B1109000F10E066246394712C08
:103E7000601A710A88279927801B910BFC01EE0FAD
:103E8000FF1FFE87ED87A701400F511F21E0B601FC
:103E900084EE96E00E94E42AA701401B510B21E02A
:103EA000B60184EE96E00E94E42AB601600F711F0D
:103EB00021E0A70184EE96E00E94E42AB601601B8F
:103EC000710B21E0A70184EE96E00E94E42A15011F
:103ED000F9E02F0E311C9501295F3F4F38872F8362
:103EE000188A1F8641E050E05A8B498BC4018A1919
:103EF0009B099C8B8B8BEF85F889E017F1070CF001
:103F000073C077FC09C001501109AD85BE851296BA
:103F1000BE87AD876A0E7B1EEF85F8893196F88BD8
:103F2000EF8729893A892E5F3F4F3A8B298B620EA2
:103F3000731E21E05701A00EB11EA501B10184EE50
:103F400096E00E94E42A21E0A5016F81788584EE45
:103F500096E00E94E42A21E05701A01AB10AA501C7
:103F6000B10184EE96E00E94E42A21E0A5016F8170
:103F7000788584EE96E00E94E42AAB88BC88A20C87
:103F8000B31C21E0A5014601800E911EB40184EE10
:103F900096E00E94E42A21E0A5015601A01AB10A88
:103FA000B50184EE96E00E94E42A4B895C898F81FA
:103FB0009885480F591F5A87498721E0B40184EE3C
:103FC00096E00E94E42A21E049855A85B50184EEF5
:103FD00096E00E94E42A9FEF291A390AAF81B8853A
:103FE0001197B887AF8387CF2B813C81265F3F4FE6
:103FF0003C832B834D815E81465F5F4F5E834D83A3
:104000005AE0450E511C2D5C324009F0ACCEAB8518
:10401000BC8516968C911697882321F18D919C91E1
:1040200011972091730130917401821B930B1296AA
:104030006D917C9113972091750130917601AC01BF
:10404000415051094F37510568F4621B730B9B01B6
:10405000215031092F33310528F420E04EEF5CE088
:104060000E94FC29EB85FC853796FC87EB87E3579C
:10407000F14069F68091D7028770843088F5E0902E
:104080007501F090760100917301109174016091B7
:10409000D4027091D5026E197F098091D20290915D
:1040A000D3022091CF0244E051E1801B910B0E948A
:1040B000C12A2091CF02220F220F8091D002280F17
:1040C0006091D4027091D5026E197F098091D2025D
:1040D0009091D30242E05DE0801B910B0E94FC298D
:1040E00021E030E041E060E086E50E94CE2510E06E
:1040F0008091D602181778F4812F869520E046E04B
:1041000052E160E070E03AE0839FC00111240E9418
:10411000F6291F5FEDCF10E08091D6028695181723
:1041200068F421E046E052E160E070E0AAE01A9F06
:10413000C00111240E94F6291F5FEECF10E020E09D
:1041400030E080E0F901E057FE4F948191118F5FDC
:104150002B5F3F4F29313105A9F7181770F4B9E0EB
:104160001B9FC001112422E046E852E160E070E0AC
:1041700088960E94F6291F5FE2CF81112FC080919F
:104180000001882391F023E046E852E160E070E00E
:104190008DE290E00E94F62924E046E852E160E0DA
:1041A00070E086E390E00E94F62925E046E852E1BF
:1041B00060E070E081E490E00E94F62926E046E8A5
:1041C00052E160E070E08AE490E00E94F62920E08D
:1041D00030E040E061E084E40E94CE258091DA0284
:1041E0008823A9F010E08091DC02181780F420E009
:1041F00046E053E167E070E0812F90E00E94F629ED
:104200001F5FF1CFD6018C9189258C93F8CC6996EC
:104210000FB6F894DEBF0FBECDBFDF91CF911F91D7
:104220000F91FF90EF90DF90CF90BF90AF909F9055
:104230008F907F906F905F904F903F902F90089558
:104240001092C2011092C10186E08093CD021092BB
:10425000AD011092AE011092AF011092B001109218
:10426000AA011092A901EEECF2E0118285E08087AC
:1042700011868AE0838381E08487158616860895F7
:104280001092AC011092AB011092C2011092C101C8
:104290001092AD011092AE011092AF011092B001D8
:1042A0001092AA011092A901EEECF2E0118285E0D1
:1042B000808711868AE0838381E08487158616864D
:1042C00086E08093CD0208951092BE0181E0809334
:1042D000BD018091BB019091BC01853191055CF4D9
:1042E00004969093BC018093BB018091BA018450E5
:1042F0008093BA0108958091C0018F5F8093C001BF
:1043000008958091E7069091E80683709927892B9C
:1043100029F48091C3018F5F8093C3018091C30111
:10432000893038F08091C0018F5F8093C001109276
:10433000C30108958091B8018823B9F0815080931A
:10434000B8018091AD019091AE01A091AF01B09103
:10435000B0010596A11DB11D8093AD019093AE01F2
:10436000A093AF01B093B00108958091C1019091E5
:10437000C2018138910524F0809106018E3031F41C
:104380008091C0018F5F8093C00108958BE080937E
:10439000CD021092C00108958EEC9FEF9093BC0166
:1043A0008093BB018AE98093BA018091C101909109
:1043B000C201019721F0809106018D3049F41092DD
:1043C000BE0181E08093BD011092BF0184E00AC06C
:1043D00081E08093BE011092BD011092BF018091D7
:1043E000C0018F5F8093C0010895909106019E30B7
:1043F00019F0E091C10102C0E091AB01F0E031970A
:10440000EE0FFF1FEE0FFF1FE80FF11DE45FFC4EE4
:10441000849128E0829FC001112408958091E706CD
:104420009091E8066EE170E00E948636892B31F4A7
:104430009091BF0181E089278093BF018CE00E94A9
:104440003A2F882339F081E08093CD021092C00189
:104450001092BF01089520E042E256E260E070E071
:1044600080E290E00E94FC2921E042E256E260E214
:1044700070E080E290E00E94FC298CE00E943A2FDC
:10448000882319F081E08093CD0208958091C301C3
:104490008F5F8093C30120E04CE754E264E070E05A
:1044A00082E290E00E94FC298091C301893728F0C4
:1044B0001092C30181E08093CD02089520E046E987
:1044C00059E160E070E08EE190E00E94FC2920E07C
:1044D0004CE759E160E070E08CE590E00E94FC2937
:1044E00020E046E059E168E270E085E290E00E9459
:1044F000FC298CE00E943A2F882361F088E08093A9
:10450000CD0220E040E358E160E270E086E190E017
:104510000C94FC2908950F931F93CF93DF9380E5AC
:1045200090E00E940D36C82F8091C501C81306C0C7
:1045300088E590E00E940D368C1741F08CE0809366
:10454000CD02DF91CF911F910F9108951092AD018F
:104550001092AE011092AF011092B0011092AA0118
:104560001092A9011092CF0285E08093D60210929A
:10457000D7028AE08093D10281E08093DA02109220
:10458000DB021092DC0281E590E00E940D36809300
:10459000AB0182E590E00E940D368093AC018091E2
:1045A000AB019091AC019093C2018093C1010DEADF
:1045B00011E0C3E5D0E0CE010E940D36F8018193F1
:1045C0008F012196C735D105B1F787E590E00E94AC
:1045D0000D368093D60286E0B2CF109294011092ED
:1045E000990110929E011092A3011092A8011092BD
:1045F0007B011092830110928B0180E090E0FC011E
:10460000E352FE4F17820A96803F9105C1F78091D1
:10461000AB019091AC019C012F5F3F4F3093AC01F7
:104620002093AB01209106012E3051F060E270E042
:104630000E949A3601969093AC018093AB010EC014
:104640000E94993520E230E040E050E00E9423369D
:104650006F5F7F4F7093AC016093AB018091C1019C
:104660009091C20101969093C2018093C101109272
:104670008F011092C0011092C30187E08093CD0298
:1046800008958F929F92AF92BF92EF92FF920F93F5
:104690001F93CF93DF9300D000D0CDB7DEB78091CA
:1046A000E7069091E8066EE170E00E948636892B5D
:1046B00031F49091BF0181E089278093BF018CE0A4
:1046C0000E943A2F882309F401C188E08093CD022B
:1046D0001092C0011092BE011092BD011092BF0154
:1046E0008EEC9FEF9093BC018093BB018AE980938D
:1046F000BA0180E00E94F5219093D3028093D20208
:1047000081E00E94F5219093D5028093D40283E04A
:104710000E94F5218C0182E00E94F5219093B20164
:104720008093B1011093B4010093B30101151105F9
:10473000A1F0803F21E0920741F0003F110541F0D8
:10474000892B49F403E010E008C001E010E005C047
:1047500002E010E002C000E010E00093B601109209
:10476000B5018FEF8093B8018093B90101E011E0AA
:1047700025E0822E912CA12CB12C35E0F32EF00EE9
:104780000E949935D801EC90A50194010E9423362E
:10479000E62FF0E0EF5FFE4F8081D8018D938D0111
:1047A000E082FA12EDCF809106018E3009F457C0F5
:1047B0006091C50180E590E00E9415366091AB01E3
:1047C0007091AC01615071097C836B8381E590E04D
:1047D0009A838983CE0101960E948E166C8182E5B0
:1047E00090E09A838983CE0101960E948E169DEAFD
:1047F000E92E91E0F92E03E510E0F70161917F01C8
:104800001A830983CE0101960E948E160F5F1F4FF7
:104810000735110591F76091D6021A830983CE01FD
:1048200001960E948E166091C50188E590E00E9475
:1048300015368091C1019091C20160E870E00E943C
:104840009A369C012150310937FF02C0215E3F4F4B
:1048500085E0359527958A95E1F72E5F01C025E023
:104860004091AB015091AC01415051093AE0349F65
:10487000C001359F900D1124A0E9B1E030E051E076
:10488000321721F1432F440FFC01E40FF11DE45FC7
:10489000FA4EE49168E0E69FF00111241196FC9332
:1048A000EE934F5FFC01E40FF11DE45FFA4EE491DB
:1048B00048E0E49FF00111241396FC93EE931297C5
:1048C00014965C9314973F5F1596DACF0F900F9074
:1048D0000F900F90DF91CF911F910F91FF90EF906C
:1048E000BF90AF909F908F9008958091C4018F5F8B
:1048F0008093C401873140F08091C3018F5F809322
:10490000C30186E18093C4018091C301863018F011
:1049100085E08093C301089520E04AE852E260E018
:1049200070E080E090E00E94FC2920E044EF51E23A
:1049300060E270E08EE390E00E94FC2920E04EE30C
:1049400058E260E070E082E490E00C94FC29AF92C1
:10495000BF92CF92DF92EF92FF920F931F93CF936C
:10496000DF930E948C2400E010E0CFE7D0E080913C
:10497000C4019E01281B3109C901800F911F0E94AB
:10498000452F085F1F4F0831110589F7C0910701B6
:10499000C23021F482E690E00E94452F89E1E82EA2
:1049A000F12C02E010E0AC2EB12C90E8C92ED12CF5
:1049B0008091C40125E0200F0A151B0539F047E45A
:1049C0005AE2B701D601A81BB1090BC0F601E81BDA
:1049D000F1099091C30147E45AE2B701DF01A91B35
:1049E000B109CD010E94FC290F5F1F4FB9E0EB0E0A
:1049F000F11C05301105E1F680E10E943A2F882371
:104A000011F0C43090F180E80E943A2F882321F001
:104A100080910701833078F584E00E943A2F882343
:104A200061F01092C3011092C40180910701865F6A
:104A30008093CD02809306010CC088E00E943A2F3B
:104A4000882339F01092C3011092C40181E0809351
:104A5000CD02DF91CF911F910F91FF90EF90DF90EA
:104A6000CF90BF90AF900C947524CF5FC093070197
:104A70001092C301C8CF8150809307011092C301E7
:104A8000CBCFAF92BF92CF92DF92EF92FF920F9374
:104A90001F93CF93DF930E948C2400E010E0CFE7B8
:104AA000D0E08091C4019E01281B3109C901800F0B
:104AB000911F0E94452F085F1F4F0831110589F78C
:104AC000C0910701C23021F482E690E00E94452F98
:104AD00089E1E82EF12C02E010E0AC2EB12C90E838
:104AE000C92ED12C2EEF200F8091C4010A151B0571
:104AF00039F047E45AE2B701D601A81BB1090BC04F
:104B0000F601E81BF1099091C30147E45AE2B701AD
:104B1000DF01A91BB109CD010E94FC290F5F1F4FC6
:104B2000B9E0EB0EF11C06301105E1F680E10E94C0
:104B30003A2F882311F0C53028F180E80E943A2FDF
:104B4000882321F080910701833010F58CE00E94CA
:104B50003A2F882359F01092C3011092C40180911A
:104B600007018093CD0282E080930701DF91CF910E
:104B70001F910F91FF90EF90DF90CF90BF90AF907B
:104B80000C947524CF5FC09307011092C301D5CF59
:104B90008150809307011092C301D8CF6F927F920A
:104BA0008F929F92AF92BF92CF92DF92EF92FF923D
:104BB0000F931F93CF93DF93CDB7DEB72A970FB62E
:104BC000F894DEBF0FBECDBFF82EE62E742E213036
:104BD000310571F02230310521F1232BB9F5809197
:104BE000B8014AE08E010F5F1F4FB80190E022C06C
:104BF0006091AD017091AE018091AF019091B001D3
:104C00002AE08E010F5F1F4FA8010E94B235F80104
:104C100001900020E9F73197E01BF10B8E2E06E0A2
:104C200014C04AE08E010F5F1F4FB8018091C1018F
:104C30009091C2010E94A735F80101900020E9F788
:104C40003197E01BF10B8E2E03E00E1B912C002EF2
:104C5000000C110BCE2CD12CAF2CB12C892D90E057
:104C6000801791077CF521E07216D9F0721670F06A
:104C700032E0731225C020E040E950E2B601C501E0
:104C80003AE0939E800D911D112418C0880F991F42
:104C9000880F991F20E044ED51E2B6018A0D9B1D5B
:104CA0000DC020E042E351E2B601C50137E0939E1A
:104CB000800D911D11240E94F62902C00E94FC293A
:104CC0009394CCCF8F2D90E06801CC0CDD1CCC0CE4
:104CD000DD1CC80ED91E27E0209F5001219FB00C7B
:104CE0001124A80EB91E4AE0409F9001419F300D4B
:104CF00011248901080F191F612C082C000C990838
:104D0000F12C862D90E088159905CCF5E1E0F0E0D6
:104D1000EC0FFD1FE80FF91F208121331CF02053F9
:104D20002A3008F020E031E07316C9F0731668F0FD
:104D300082E0781222C040E950E2B701C8013AE0AF
:104D4000639E800D911D112416C0880F991F880F36
:104D5000991F44ED51E2B7018C0D9D1D0CC042E33B
:104D600051E2B701C50137E0639E800D911D11240A
:104D70000E94F62902C00E94FC296394C2CF2A96A1
:104D80000FB6F894DEBF0FBECDBFDF91CF911F915C
:104D90000F91FF90EF90DF90CF90BF90AF909F90DA
:104DA0008F907F906F900895E091C001F0E0EE0F3A
:104DB000FF1FEA5DF74E85919491FC01099520E073
:104DC0004CE757E168E070E086E190E00E94FC2942
:104DD00021E030E042E060E284E20E94CE25809152
:104DE000BF01882349F020E044E457E168E370E024
:104DF00085E290E00C94FC290895E091C001F0E078
:104E0000EE0FFF1FEA5DF74E85919491FC01099525
:104E10008091060120E08E3039F444E157E163E0EF
:104E200070E089E290E006C048EE56E163E070E091
:104E30008BE290E00E94FC2920E040E358E16FE023
:104E400070E08BE090E00E94FC2921E030E042E03D
:104E500062E283E20E94CE258091BF01882349F05F
:104E600020E044E457E165E370E085E290E00C94D3
:104E7000FC290895E091C001F0E0EE0FFF1FE6521B
:104E8000F94E85919491FC0109958091BE0188238A
:104E9000B9F020E046EB56E160E170E080E290E09E
:104EA0000E94FC2920E030E041E060E18EE40E94B5
:104EB000CE2521E030E042E064E284E20E94CE258B
:104EC0008091BD018823A1F120E04CE456E168E126
:104ED00070E08091BB019091BC010E94FC298091FF
:104EE000BF018823E9F08091060120E08E3039F47B
:104EF00044E157E168E070E089E290E006C048EEE6
:104F000056E168E070E08BE290E00E94FC2920E02E
:104F100044E457E160E370E085E290E00E94FC2900
:104F200022E030E042E068E18091BA010C94CE25A5
:104F30000895FC01A3E0F695E795AA95E1F79B019A
:104F4000287F3327E20FF31FF695E7952091AB01F9
:104F50003091AC012150310944E0220F331F4A95B2
:104F6000E1F7E20FF31FE057F14E249130E0AC017E
:104F70004870552783FD03C0EFEFF0E002C0EFE07B
:104F8000F0E02E233F23452B11F444E001C040E024
:104F9000FB01E770FF2753E0EE0FFF1F5A95E1F783
:104FA00087709927E80FF91F02C0359527954A9514
:104FB000E2F766E0220F331F6A95E1F7E20FF31F75
:104FC000E057F54E849108950895CF92DF92EF92C5
:104FD000FF920F931F93CF93DF936C017A018B01A4
:104FE000C0E0D0E0CE15DF0589F0D8016D918D01CC
:104FF000D601ED91FC910190F081E02DC60109955B
:10500000892B11F47E0102C02196ECCFC701DF91FC
:10501000CF911F910F91FF90EF90DF90CF90089567
:105020003FB7F8948091D1019091D201A091D30122
:10503000B091D40126B5A89B05C02F3F19F0019669
:10504000A11DB11D3FBFBA2FA92F982F8827820F0E
:10505000911DA11DB11DBC01CD0142E0660F771F5E
:10506000881F991F4A95D1F708958091E102E09138
:10507000DF02F091E002882349F0CF01029690937D
:10508000E0028093DF02859194910895CF0102960A
:105090009093E0028093DF02808191810895809156
:1050A000C60108951092C6013E983F9808953E9A11
:1050B0003F9A81E08093C60108950E94B4368F9292
:1050C0009F92AF92BF92CF92DF92EF92FF926B01CD
:1050D0007C010E9410284B015C01C114D104E10441
:1050E000F104F1F00E941028DC01CB018819990924
:1050F000AA09BB09883E9340A105B10570F321E0E0
:10510000C21AD108E108F10888EE880E83E0981EE3
:10511000A11CB11CC114D104E104F10419F7DDCFC5
:10512000FF90EF90DF90CF90BF90AF909F908F90C7
:105130000895BC0180E090E00C945F281F920F92CC
:105140000FB60F9211242F933F938F939F93AF939A
:10515000BF938091D5019091D601A091D701B091D4
:10516000D8013091D00123E0230F2D3720F4019690
:10517000A11DB11D05C026E8230F0296A11DB11D7A
:105180002093D0018093D5019093D601A093D701AD
:10519000B093D8018091D1019091D201A091D30117
:1051A000B091D4010196A11DB11D8093D1019093BE
:1051B000D201A093D301B093D401BF91AF919F913D
:1051C0008F913F912F910F900FBE0F901F901895C8
:1051D000CF92DF92EF92FF920F931F93CF93DF93C3
:1051E0000E943528811520E8920761F480917100B2
:1051F0008D7F80937100109291004698479810928D
:10520000C9018BC021E02093C901813020E89207B9
:1052100051F48091DD029091DE029093E002809340
:10522000DF020E94352897FD05C02091C801222386
:1052300009F43FC02091C70121113BC021E0209318
:10524000CA01EC01DF77209769F481E08093CB01FC
:1052500046983FE9C32E3FE0D32EE12CF12CCAEF54
:10526000D0E014C08E0120E030E060E472E48FE012
:1052700090E0A90198010E94233669017A0181E03A
:10528000C81AD108E108F1081092CB01E091E206BA
:10529000F091E3060995811103C081E08093CB0171
:1052A0008091CA018823B9F18091CB01811133C06B
:1052B00003C01092CA01C5CF46992DC0479A0E94DB
:1052C0003528009771F09C01DE010E947736DC01E1
:1052D000CB0129E0B595A795979587952A95D1F7A4
:1052E00003C08FEF9FEFDC01109290002AE0209323
:1052F0009100D0929900C09298008093CC01909335
:10530000CD01A093CE01B093CF0180917100826056
:105310008093710002C04798D2CFDF91CF911F9147
:105320000F91FF90EF90DF90CF9008951F920F9212
:105330000FB60F9211242F933F934F935F936F9368
:105340007F938F939F93AF93BF93EF93FF9380913E
:10535000CC019091CD01A091CE01B091CF01892BCC
:105360008A2B8B2B81F18091CB0181110BC098B1DD
:1053700080E4892788B98091CA01882319F088B10F
:10538000805888B98091CC019091CD01A091CE0137
:10539000B091CF01181619061A061B06B4F48091B5
:1053A000CC019091CD01A091CE01B091CF01019798
:1053B000A109B1098093CC019093CD01A093CE01B6
:1053C000B093CF0102C00E94E828FF91EF91BF91F6
:1053D000AF919F918F917F916F915F914F913F918D
:1053E0002F910F900FBE0F901F9018950F9303E011
:1053F0000E94D62B0F9108950F930AEF0E94D62B8F
:105400000F910895EF92FF920F931F93CF93DF9325
:1054100000D0CDB7DEB70E948C2400E010E08FE70B
:10542000E82EF12C8091C4019701281B3109C90194
:10543000800F911F0E94452F085F1F4F08311105F3
:1054400089F780E10E943A2F882321F00E94572893
:105450001092C30180E80E943A2F882321F00E9415
:1054600052281092C3018CE00E943A2F882389F0C1
:105470001092C3011092C4016091C60182E090E0D5
:105480009A838983CE0101960E948E1681E08093D3
:10549000CD028091C40100E810E0081B110924E04E
:1054A00047E45AE269E170E0C8010E94FC2980915A
:1054B000C601882381F025E047E45AE262E270E009
:1054C000C8010E94FC298091C30126E047E45AE20A
:1054D0006BE270E00FC026E047E45AE26BE270E056
:1054E000C8010E94FC298091C30125E047E45AE2EB
:1054F00062E270E0F801E81BF109CF010E94FC298B
:105500000E9475240F900F90DF91CF911F910F9102
:10551000FF90EF90089520E04EE358E260E070E0E5
:105520008EE190E00E94FC2920E044E258E260E035
:1055300070E08CE590E00E94FC2920E041E659E211
:1055400061E270E080E390E00E94FC2920E04AE400
:1055500059E261E270E086E190E00E94FC2920E0DF
:1055600048E359E26FE270E08BE190E00E94FC2991
:105570008CE00E943A2F882319F081E08093CD02BD
:1055800008950F930BEF0E94D62B0F9108958FB1C2
:105590002CB193B130E02095309520743327A901C8
:1055A00023E0559547952A95E1F7292F30E020957E
:1055B0003095207133273595279535952795242BE0
:1055C0008095807F822B089560387105D0F4403437
:1055D0005105B8F4EBE6FBE280E1849FD001A078AE
:1055E0001124A60F4770E40FF11D8491AE51BD4FF9
:1055F000222319F06C91862B03C080956C91862331
:105600008C9308957F928F929F92AF92BF92CF9288
:10561000DF92EF92FF920F931F93CF93DF936C0172
:105620005B017A0180910F01882309F46BC080919E
:10563000DC01882309F466C08091DA0180FF05C08F
:105640008091E00082608093E000E70110E00AEFC3
:1056500083E0982E90E4792E2AE3822E209709F495
:1056600048C08FB7F8949092E9009091E80095FFB8
:1056700006C09091F200272D291B922F01C090E0C7
:105680008FBF91110AC0015009F43CC061E070E085
:1056900080E090E00E945F28E1CF292F30E0C21720
:1056A000D3070CF49C2F8FB7F8949092E9002091C7
:1056B000E80025FF1CC0292F30E0C21BD30BF501E9
:1056C000915020F041914093F100FACFA20EB31E09
:1056D000112319F08092E80009C09091E80095FD2F
:1056E00006C08092E80011E0209709F010E08FBF1B
:1056F000B5CF1111B6CF5D9884E68093D9011E1401
:105700001F0444F081E090E0F6019383828380E0FF
:1057100090E001C0C701DF91CF911F910F91FF90E1
:10572000EF90DF90CF90BF90AF909F908F907F9041
:10573000089580E0E2EEF2E081118FEF0024819382
:105740008193819381930394D1F708958091E2022C
:105750008EBDE3EEF2E081910DB407FEFDCF8EBD6C
:1057600086E0E23EF807B9F70DB407FEFDCF0895D5
:105770009C01E1E7F0E090819D7F90831092E1022F
:10578000E2E5F7E0F093E002E093DF02F093DE025F
:10579000E093DD023183208384E190E09383828370
:1057A00080E090E8958384830C94E8286F927F9240
:1057B0008F929F92AF92BF92CF92DF92EF92FF9221
:1057C0000F931F93CF93DF9300D000D0CDB7DEB7F8
:1057D000DC014115510509F4F2C1FA011491319629
:1057E00094916A01F2E0CF0ED11CE12EF12C22231C
:1057F00009F1492F469546954695E42FF0E041E0A2
:1058000050E0892F877011F440E050E04E0F5F1F89
:10581000E49EF001E59EF00DF49EF00D112403309E
:1058200011F4EE0FFF1F2E9FA0012F9F500D11248A
:10583000C40ED51E0F3F09F402E0AD014E0D5F1DF1
:10584000141615060CF0BBC1A038B1050CF0B7C199
:105850009B01290F311D121613060CF0B0C16034E4
:1058600071050CF0ACC1C114D10409F4A8C19B01AD
:1058700077FF04C022273327261B370B322F3770C0
:10588000FB0177FD379623E0F595E7952A95E1F73B
:105890002E2F77FF07C0332329F02FEF2E0F88E03C
:1058A000831B382FB7FF05C0662777276A1B7B0B42
:1058B00002C060E070E04038510524F050E85A1B07
:1058C000952E01C0912E961AA22E022E000CBB0816
:1058D0002F3F1CF48A2D809501C080E041E0592FB4
:1058E000577009F440E0969596959695940FA90EF9
:1058F000B11C49E0A416B10414F098E0921B981B67
:10590000280F40E82403A00DB11D1124A60FB71FD6
:10591000819F600D711D11243601660E771E41E0D6
:1059200050E06A01032E02C0CC0CDD1C0A94E2F7A1
:10593000033009F400C1A0F4013009F4B1C0023011
:1059400009F03DC18FEF8C9DB0018D9D700D11242C
:10595000609570957C836B838C80492F420F29C0A2
:105960000A3F31F00B3F09F02AC1492F420F84C092
:10597000492F420F4FC0F301E00FF11FE491EC9D5E
:105980005001ED9DB00C1124BA82A98227FD05C0FB
:10599000FC0150815623A52AA082311113C00F5F4C
:1059A0001F4F0196091538F32F5F6E0C7F1CA0580E
:1059B000BF4F241709F403C1CD018E519D4F00E064
:1059C00010E0F0CF27305CF7FC01E058FF4F50812A
:1059D0005821BA805B295083E2CFF301E60FF71F0D
:1059E000E491EC9D8001ED9D100D11241A83098333
:1059F00027FD04C0FC015081052B0083311113C029
:105A00006F5F7F4F0196691540F32F5F6E0C7F1C0F
:105A1000A058BF4F241709F4D2C0CD018E519D4F1D
:105A200060E070E0F0CF27305CF7FC01E058FF4FFA
:105A300010815A81512B5083E3CFF301E00FF11F06
:105A4000E491EC9DC001ED9D900D11249A83898312
:105A500027FD05C08095FB0190818923808331114A
:105A600014C00F5F1F4F6F5F7F4F091530F32F5F1B
:105A70006E0C7F1CA058BF4F241709F4A0C0BD01B5
:105A80006E517D4F00E010E0F0CF273054F7FB015E
:105A9000E058FF4F8A818095908189238083E1CFF0
:105AA000892E820EA301CB0186199709281509F4C6
:105AB00086C0BD016E517D4F5B0100E010E009150D
:105AC000A0F5F801E80FF91FE40FF51FE491EC9D34
:105AD000B001ED9D700D1124609570957C836B83F2
:105AE000FA01E00FF11FE491EC9D3001ED9D700C87
:105AF00011247A82698227FD05C0F5017081672330
:105B0000662A6082332359F027304CF4F501E058BF
:105B1000FF4F70816C8167237A81672B60830F5FF1
:105B20001F4FFFEFAF1ABF0ACACF2F5F4E0D5F1D89
:105B3000A058BF4FBBCFA92CB12CF301E60FF71F24
:105B4000AE51BD4F60E870E06A197B09EA18FB08A6
:105B50008701000F111F592D492F792CE32ECF9368
:105B6000DF93ED01EF96EF9622968590A590EE20BB
:105B700059F08C9C4001AC9C500127302CF4F880EB
:105B8000B094FB20F928F99222233AF0FC90A094DB
:105B9000FA20F828FD920C94CE2D11965A9529F7EB
:105BA0004A9551F0572D23951124E00FF11DA60FB2
:105BB000B11DC60FD11DD9CFDF91CF9111240F9008
:105BC0000F900F900F90DF91CF911F910F91FF9049
:105BD000EF90DF90CF90BF90AF909F908F907F908D
:105BE0006F9008959091D70291111BC09091D602A9
:105BF000980F9093D60287FF07C08CE38093D7025B
:105C000080E793E00E94B82B8091D602893020F083
:105C100088E08093D6020895811103C089E08093C3
:105C2000CD0208956F927F928F929F92AF92BF9212
:105C3000CF92DF92EF92FF920F931F93CF93DF9358
:105C40007C016B01142F5901CDEDD1E0F60180806C
:105C50009180F7016080718000E120E1A401B3012F
:105C6000CE010E94AE16882339F188819981681689
:105C7000790629F42A813B8182169306E9F0F50121
:105C80002081112349F0121614F4409703C02223F7
:105C900089F04096F7010CC0121624F48A819B818A
:105CA000409705C0222331F08A819B814096F601FE
:105CB00091838083F50110822A96F2E0CD3CDF07C4
:105CC00029F6DF91CF911F910F91FF90EF90DF9018
:105CD000CF90BF90AF909F908F907F906F900895DE
:105CE0002F923F924F925F926F927F928F929F92EC
:105CF000AF92BF92CF92DF92EF92FF920F931F93DA
:105D0000CF93DF9300D01F92CDB7DEB75C016B015C
:105D10003901FC0100811181C8018770992731E0A8
:105D2000892B09F430E0F6018081918187709927F1
:105D300021E0892B09F420E017FF02C0095F1F4F03
:105D4000E3E015950795EA95E1F77801FFEFEF1A83
:105D5000FF0AF3E0EE0CFF1CFA95E1F7232E312C3D
:105D6000422E512CF5018081918197FD079623E009
:105D7000959587952A95E1F70296820D931D081750
:105D800019070CF061C0F6018081918197FD07969B
:105D90009C0173E0359527957A95E1F73B832A833B
:105DA000470138E1831A9108F6018081918197FDBE
:105DB000079633E0959587953A95E1F70296840D1D
:105DC000951D2A813B8128173907C4F56A817B819B
:105DD000C80149830E9499272A813B812F5F3F4F49
:105DE00049818B3040F1F3018081442361F087FFCA
:105DF00004C0F501F182E0821CC08823D1F0F501D6
:105E00009182808216C087FF07C0C90163E0880FB6
:105E1000991F6A95E1F70AC0882359F08A819B810E
:105E200053E0880F991F5A95E1F74097F601918347
:105E30008083F30110823B832A83B6CF0F5F1F4F0D
:105E400038E0E30EF11C8ECF0F900F900F90DF9192
:105E5000CF911F910F91FF90EF90DF90CF90BF9067
:105E6000AF909F908F907F906F905F904F903F90FA
:105E70002F9008952091EA06282329F49091E906AD
:105E8000982381E009F480E008950F9302E020E078
:105E900040E55CE269E170E00E94D62B0F91089525
:105EA000FC018091DC01811103C08FEF9FEF089509
:105EB0009FB7F89482E08093E9002091F20030E0EF
:105EC0001216130614F421E030E02115310559F0C3
:105ED000289884E68093DB018091F1008083809193
:105EE000F200882319F09FBFC90108958BE68093C3
:105EF000E800F9CF8091FA0681110DC082E080930D
:105F0000F60684E08093F7061092F9061092F806E0
:105F100081E08093FA0686EF96E00895CF93DF93B1
:105F20001F92CDB7DEB76983DC01ED91FC91028051
:105F3000F381E02D41E050E0BE016F5F7F4F099596
:105F40000F90DF91CF91089583E08093E9008091D5
:105F5000F200882319F08AE38093E8000895FC0199
:105F60008485958597FD0BC09FB7F89482E0809358
:105F7000E9008091F2009FBF90E0019608959FB7DD
:105F8000F89482E08093E9008091F2009FBF90E056
:105F90000895409164075091650720916207309100
:105FA000630742175307B4F49091E8009570E1F34A
:105FB0009091E80092FD19C08093F10080916407F0
:105FC0009091650701968F739927892B19F48EEFAD
:105FD0008093E80080916407909165070196909303
:105FE00065078093640781E0089580E00895DF925B
:105FF000EF92FF920F931F93CF93DF93D82E8A01D6
:106000007B01E40EF51EEB01CE15DF0571F0D7FE26
:1060100003C0FE01849101C088810E94C92F21968E
:106020008111F2CF8FEF9FEF01C0C801DF91CF91B7
:106030001F910F91FF90EF90DF900895615030F025
:106040002091F100FC0120830196F8CF289884E686
:106050008093DB0108950F931F93CF93DF931F92DB
:10606000CDB7DEB78C01FC018485958597FF0EC006
:10607000CE0101960E94502F019719F4298130E03A
:1060800002C02FEF3FEFF80135872487F8018485A0
:1060900095850F90DF91CF911F910F910895CF9328
:1060A000DF931F92CDB7DEB7FC018485958597FD00
:1060B00005C02FEF3FEF358724870BC0CE01019637
:1060C0000E94502F019719F4898190E002C08FEF50
:1060D0009FEF0F90DF91CF9108950F931F93CF9370
:1060E000DF931F92CDB7DEB782E0898342E450E0B0
:1060F0006AE57CE280E80E94F72F0E947A2FDC019B
:1061000012960D911C9113970115110569F0D80194
:10611000ED91FC910280F381E02DBE016F5F7F4F16
:10612000C801099597FF07C089810F90DF91CF9132
:106130001F910F910895F80100851185E5CF1F92F9
:106140000F920FB60F9211248F939F938091E100CD
:106150009091E100937F9093E10083FF0FC0109234
:10616000E90091E09093EB001092EC0092E39093A1
:10617000ED001092DC0198E09093F00082FF20C0C7
:1061800093E09093E9009091F200992319F09AE33B
:106190009093E8009091D901992339F09091D90119
:1061A00091509093D901992389F19091DB01992322
:1061B00039F09091DB0191509093DB01992341F1EB
:1061C00084FF10C08091E2008E7E81608093E200A7
:1061D0008091E1008F7E8093E1008091DA018E7ED4
:1061E000806111C080FF16C08091E2008E7E8061C8
:1061F0008093E2008091E1008E7E8093E1008091A7
:10620000DA018E7E81608093DA0104C05D9ACDCF81
:10621000289AD6CF9F918F910F900FBE0F901F900D
:1062200018951F920F920FB60F921124CF92DF9202
:10623000EF92FF920F931F932F933F934F935F9390
:106240006F937F938F939F93AF93BF93EF93FF933E
:10625000CF93DF93CDB7DEB76C97DEBFCDBF109283
:10626000E9008091E80083FFEDC168E0CE0145962A
:106270000E941E3082EF8093E8008D8987FF05C061
:106280009091E80090FFFCCF03C09EEF9093E80050
:10629000982F907609F0C6C09E892F89188D91118C
:1062A0000CC0803829F4809161078093F10002C00E
:1062B0001092F1001092F10048C1422F50E0512B92
:1062C000913051F4811141C14130510509F03DC176
:1062D000809161078D7F0BC0933061F4811135C1CE
:1062E0004130510509F031C180916107826080938E
:1062F00061072BC1953041F48091E80080FFFCCF0D
:1063000020682093E30021C1963009F05FC0EB8C38
:10631000FC8C1092E900109265071092640712300D
:1063200091F510926307109262070E946D3099E018
:10633000BE016F5F7F4FDB01E92F1D92EA95E9F700
:1063400099831A8391E09E8390EA98879AEF9987C0
:106350002091640730916507275F3F4F3C832B8373
:106360008D831092E9001092650710926407F092F5
:106370006307E092620749E050E080E00E94F72F57
:106380000E946D30E2C0F0926307E09262070E94C3
:106390007A2FDC011296ED90FC901397E114F10432
:1063A00009F4C0C0D701ED91FC910480F581E02D86
:1063B000BE016B5E7F4FC7010995009719F00CF085
:1063C000C4C0C7C0F701E084F184E8CF973009F476
:1063D000C0C0983021F481E08093F100B6C09930BC
:1063E00009F0B3C0837009F0B4C0E1E4F1E081E0EA
:1063F00021E036E39081992361F08093E9002093B6
:10640000EB0091919093EC003093ED008F5F87301B
:1064100089F78EE78093EA001092EA008F898093D3
:10642000DC0193C08B8D9C8D1092E9001092650762
:10643000109264079093630780936207898D81119E
:1064400056C08E899D89913A59F4813209F081C0F4
:1064500047E050E068E071E080E00E94F72F75C0EF
:10646000913209F076C0833289F4888D90E0982FBC
:1064700088272F89822BA0E0B0E0809310019093B1
:106480001101A0931201B09313015FC0803269F42F
:106490008091E80082FFFCCF67E088E091E00E94F5
:1064A0001E308BEF8093E80006C0823209F04DC0A9
:1064B0008F8980930F0180916007882319F0EEEF98
:1064C000FAE002C0E0E0F8E0809108019091090153
:1064D000A0910A01B0910B01803B9440A105B10548
:1064E00009F07BC080910F0180FF93C076C00E94AD
:1064F0007A2FDC0112960D911C911397011511054D
:1065000041F1D801ED91FC910190F081E02DBE01A7
:106510006B5E7F4FC8010995811117C0F801008596
:106520001185ECCF113009F44EC0133091F48F89EE
:10653000882309F445C0823081F440E867E08EEB9F
:106540009CE20E940E35882321F08EEF8093E800B4
:1065500079C081E28093EB0075C0813029F440E876
:106560006BE082EB9CE2EDCF833099F70E947A2FAB
:10657000DC011296ED90FC9013978E010F5F1F4F78
:106580006801E114F10479F0D701ED91FC910680E6
:10659000F781E02DB801C7010995080F111DF7011A
:1065A000E084F184EECFD8011C92F6010190002026
:1065B000E9F73197BF016C197D0940E0C601C1CFF1
:1065C0006CE97CE202C060EA7CE26115710509F2C7
:1065D000FB01449150E080E840CF0FB6F894A895B5
:1065E00080916000886180936000109260000FBE0F
:1065F000A895EE3F2AE0F20739F08091FE0A9091CB
:10660000FF0A91838083A1CF1092FF0A1092FE0AA5
:106610009CCFEE3F8AE0F80731F080819181909322
:10662000FF0A8093FE0A87E797E7918380839BE0C8
:1066300088E10FB6F894A895809360000FBE909300
:10664000600083CF6C960FB6F894DEBF0FBECDBF4F
:10665000DF91CF91FF91EF91BF91AF919F918F917A
:106660007F916F915F914F913F912F911F910F916A
:10667000FF90EF90DF90CF900F900FBE0F901F9084
:106680001895789484B5826084BD84B5816084BD9A
:1066900085B5826085BD85B5816085BD80916E00C0
:1066A000816080936E0010928100809181008260F1
:1066B000809381008091810081608093810080912E
:1066C000800081608093800080919100826080933F
:1066D0009100809191008160809391008091900061
:1066E0008160809390008091C10084608093C1009C
:1066F0008091C10082608093C1008091C10081605F
:106700008093C1008091C30081608093C300809119
:10671000C00082608093C0008091C200816080933D
:10672000C20080917A00846080937A0080917A0020
:10673000826080937A0080917A00816080937A00F1
:1067400080917A00806880937A001092DC01109228
:1067500061071092DA018091D70081608093D700A1
:1067600080EA8093D80089B5806189BD89B582604F
:1067700089BD09B400FEFDCF61E070E080E090E0EB
:106780000E945F288091D8008F7C80618093D80020
:106790008091E000807F8093E0008091E1008E7E18
:1067A0008093E1008DE08093E200559A209AEEEF0D
:1067B000FFE7859194918B3F9C4D19F481E0809384
:1067C000600781EC80937C0085B1806F85B9249847
:1067D00084B1866E84B95E9A5F988AB1806D8AB9F9
:1067E000769A6E9881B3806F81BB899880B38D70E3
:1067F00080BB80E58CBD81E08DBD85E090E00E948E
:1068000099285F9A85E090E00E9499285E985C98AC
:10681000E3E7FBE28DE08E0F94919EBD00000DB486
:1068200007FEFDCF31968E13F7CF5C9A81E88093F7
:10683000640081E08093650082E090E00E940D3664
:10684000882319F00E94572802C00E9452282E98CF
:10685000CEEEDFEF0E94C72A86FF03C02E9A2F9A42
:106860002CC0CC3F8FEFD80719F42E9A2F9805C073
:10687000C831D10511F42F9A2D980E94992B20E050
:1068800040E85BE2BE0184E190E00E94FC290E94A6
:10689000A62B8BE190E00E949928C03FEFEFDE0726
:1068A00021F48AEF90E00E9499282196C931D10500
:1068B00089F68CEB92E00E9499282D9A80E18093D2
:1068C000EB0688E28093C501C0E0D0E011E02FB76D
:1068D000F8948091D5019091D601A091D701B09103
:1068E000D8012FBF4091F0065091F1066091F20659
:1068F0007091F3062091F406222341F02091EC06DA
:10690000821B8093F5061092F4064CC084179507FD
:10691000A607B70778F4481B423008F443C083B792
:10692000817F83BF83B7816083BF889583B78E7F64
:1069300083BF38C01093F4068093EC069093ED0665
:10694000A093EE06B093EF062091EB06820F911D07
:10695000A11DB11D8093F0069093F106A093F2065D
:10696000B093F3068091E7069091E8060196909324
:10697000E8068093E7068091E9068093EA060E9484
:10698000C72A8093E9060E94992BE091CD02F0E09E
:10699000EE0FFF1FEE5CF34D85919491FC0109957C
:1069A0000E94A62B209709F492CF0E9400008FCF5F
:1069B000E2E0F7E01382128288EE93E0A0E0B0E01C
:1069C00084839583A683B7838EE291E0918380834D
:1069D0008FEF9FEF95878487E4EEF6E02EE331E0BA
:1069E000318320831582168220E127839483838359
:1069F0001486158616861786108A8FE498E290937F
:106A0000E3068093E20680E090E890935F0780932E
:106A10005E0746983E9A47983F9A0895CF92DF9234
:106A2000EF92FF920F931F93CF93DF931F92CDB7F7
:106A3000DEB7182F062FE42E862F880F8E5F9983DE
:106A40000E94C92F83E00E94C92FF12EC12E998187
:106A5000D92E8C2D8F19801798F4F601E7FE02C00D
:106A6000849101C080810E94C92F182F80E00E946C
:106A7000C92F8123FFEFCF1ADF0A8111EACF01C0AE
:106A800081E00F90DF91CF911F910F91FF90EF90D8
:106A9000DF90CF9008958F929F92AF92BF92CF9246
:106AA000DF92EF92FF92CF93DF93EC0168817981BF
:106AB0008A819B81611571058105910521F464E24C
:106AC00079ED8BE597E02DE133EF41E050E00E9456
:106AD000233649015A019B01AC01A7EAB1E40E94A7
:106AE00042366B017C01ACEEB4EFA50194010E942B
:106AF0005036DC01CB018C0D9D1DAE1DBF1DB7FFB7
:106B000003C00197A109B04888839983AA83BB83F6
:106B1000BC01CD019F77DF91CF91FF90EF90DF9087
:106B2000CF90BF90AF909F908F9008950E944B356B
:106B3000089584E191E00E944B350895609314011B
:106B40007093150180931601909317010895BB2748
:106B50004A3031F4992322F4BDE2909581959F4FFC
:106B60000C94E435BB272A3051F4992342F4BDE25A
:106B700090958095709561957F4F8F4F9F4F0C94A6
:106B8000C235BB27FA01A62F621771058105910551
:106B9000330B30FB66F0AA27660F771F881F991FFB
:106BA000AA1FA21710F0A21B63953850A9F7A05D89
:106BB000AA3308F0A95DA19336F7B111B193108201
:106BC000CA010C94FD35BB27FB015527AA27880F66
:106BD000991FAA1FA41710F0A41B83955051B9F751
:106BE000A05DAA3308F0A95DA193009779F7B111D0
:106BF000B1931192CB010C94FD35DC01FC01672FA0
:106C000071917723E1F7329704C07C916D93708383
:106C10006291AE17BF07C8F30895F999FECF92BDF0
:106C200081BDF89A992780B50895262FF999FECF4E
:106C30001FBA92BD81BD20BD0FB6F894FA9AF99A99
:106C40000FBE01960895052E97FB1EF400940E9436
:106C50003A3657FD07D00E94553607FC03D04EF454
:106C60000C943A3650954095309521953F4F4F4FB3
:106C70005F4F089590958095709561957F4F8F4FE8
:106C80009F4F08950E947736A59F900DB49F900D59
:106C9000A49F800D911D11240895B7FF0C944236D6
:106CA0000E944236821B930B0895A1E21A2EAA1B62
:106CB000BB1BFD010DC0AA1FBB1FEE1FFF1FA217AC
:106CC000B307E407F50720F0A21BB30BE40BF50BA9
:106CD000661F771F881F991F1A9469F76095709532
:106CE000809590959B01AC01BD01CF010895A29FB5
:106CF000B001B39FC001A39F700D811D1124911D90
:106D0000B29F700D811D1124911D0895AA1BBB1BFC
:106D100051E107C0AA1FBB1FA617B70710F0A61B9B
:106D2000B70B881F991F5A95A9F780959095BC01BC
:106D3000CD01089597FB072E16F4009407D077FD38
:106D400009D00E94863607FC05D03EF490958195C7
:106D50009F4F0895709561957F4F0895EE0FFF1F27
:106D60000590F491E02D099481E090E0F8940C9462
:066D7000B936F894FFCFD4
:106D76000100010203040C0300E100000000000012
:106D8600FFFFFFFF0100000000FEFDFE0002030200
:106D960001010100010200010001000000008E2F28
:106DA600022BAF2F4F302B30A42F00000000E4271A
:086DB60000C180810000000013
:00000001FF
